:100000000C9445010C9462010C94790E0C946201DD
:100010000C9462010C9462010C9462010C946201D4
:100020000C9462010C9462010C9462010C943011E6
:100030000C9462010C94D22E0C940C2F0C94352F3E
:100040000C9462010C9462010C9462010C9479335B
:100050000C94620131313356332E333700000001E6
:100060000000060000FF00000F02000C0014010158
:100070000400001450040100000000000000000013
:1000800000000000010003E8000000000000000381
:10009000E800000000000200FA0600070000FF0070
:1000A0000037060002800000000000002107101049
:1000B0000504030206100D0C0B0A2E1005040302A2
:1000C00006100D0C0B0A2E100504030206100D0C71
:1000D0000B0A2E1111111111111111111111111100
:1000E0001111111111111111111111111111110011
:1000F0000404040808080C0C0C1010101414181830
:10010000181C1C1C20202020242424282828282CCB
:100110002C2C2C30303030343434343438383838B7
:10012000383838383C3C3C3C3C3C3C3C3C3C3C1843
:10013000180B0B0C0C0B0C0B040208040C1803031B
:10014000030801010101010804040101000000008D
:1001500000000C10140808090A0B0C08080C090A06
:100160000B0C0D0E080808090A0A0A0A0A0B0C0CE7
:1001700000010405030647401D1B1C1B14133322FA
:1001800019100C080603016744332219100C0803E8
:10019000524F5200000106524F4C000002064D53D0
:1001A00054000003024D5650000004075341500014
:1001B0000005074741500000060353544150000713
:1001C00003525341500008035347500000090747AA
:1001D000475000000A0353544750000B0352534743
:1001E00050000C0352465300000D0353494F0000CA
:1001F0000E0747494F00000F0353414300001D07FE
:1002000053434F00001E0747434F00001F03434363
:100210004F0000200355463000004007554631008E
:10022000004107554632000042075546330000435F
:10023000075546340000440755463500004507552C
:100240004636000046075546370000470752554ED0
:100250000000810553544F5000800042494E000079
:100260008B0000000000000000535441545553001F
:1002700053544F5000535441525400434F4F524433
:100280000052454C00414253000011241FBECFE5EF
:10029000D8E0DEBFCDBF11E0A0E6B0E0E4EAF0E7D1
:1002A00002C005900D92A431B107D9F714E0A4E182
:1002B000B1E001C01D92AE3FB107E1F70E946401B9
:1002C0000C9451380C940000EF92FF920F931F93FF
:1002D000CF93DF93CDB7DEB724970FB6F894DEBF88
:1002E0000FBECDBF0E94360F82E00E9409110E940E
:1002F000A80F8DB18F738DB981E887BB30E020E006
:1003000018BA00000000000096B380E888BB000027
:1003100000000000B69B02C096FF2F5F3F5F3A309F
:1003200079F72A3039F560E089E090E00E94761094
:1003300060E080E090E00E9476101A82198205C089
:1003400089819A8101969A83898389819A818F5FB5
:100350009F4FB1F7C0981A82198205C089819A818E
:1003600001969A83898389819A818F5F9F4FB1F724
:10037000C09AE3CF0E94360F82E00E9409110E94CA
:100380008B0E0E948B110E94A80FAB980E94750FD4
:100390000E948B0F80E090E00E946E10843E09F472
:1003A000DBC0C0980E94F12F60E089E090E00E94DD
:1003B000761040E16DE570E080E090E00E94BB10B7
:1003C00061E08AE491E00E94761060E08BE491E0C5
:1003D0000E94761060E08CE491E00E94761060E06C
:1003E0008DE491E00E94761062E08EE491E00E943C
:1003F000761060E08FE491E00E94761060E080E586
:1004000091E00E94761060E081E591E00E94761014
:100410000E9493104DE26CE770E08DE390E00E9443
:10042000BB104DE26CE770E08AE690E00E94BB10E2
:100430004DE26CE770E087E990E00E94BB1043E07A
:1004400069EA70E084EC90E00E94BB1043E06CEA43
:1004500070E087EC90E00E94BB1040E86FEA70E02B
:100460008AEC90E00E94BB106FEF8AE591E00E9459
:1004700076106FEF8BE591E00E9476106FEF8CE5C0
:1004800091E00E9476106FEF8DE591E00E9476106A
:100490006FEF8EE591E00E9476106FEF8FE591E0AF
:1004A0000E94761060E080E691E00E94761060E0A5
:1004B00081E691E00E94761060E082E691E00E9481
:1004C000761060E083E691E00E94761060E084E6BA
:1004D00091E00E94761060E085E691E00E9476103F
:1004E00060E08DEF93E00E94761060E08EEF93E085
:1004F0000E94761060E08FEF93E00E94761060E03B
:1005000086E691E00E94761068E087E691E00E941E
:10051000761060E088E691E00E94761068E089E657
:1005200091E00E94761060E08AE691E00E947610E9
:1005300068E08BE691E00E94761081E090E00E94F6
:100540006E10EEE5F0E0E4918E1729F464EE80E0A1
:1005500090E00E947610C09A81E090E00E946E10B8
:100560000E944A2F8EE70E94A70A00E0802F806138
:100570000E94A70A802F88610E94A70A802F8460AA
:100580000E94A70A802F86600E94A70A802F84619C
:100590000E94A70A005E003649F70E9426090E94C1
:1005A000E310EE24FF24C70125E0880F991F2A9548
:1005B000E1F78D600E944010082F10E0C8010196FD
:1005C0000E946E108C83C80102960E946E108B836D
:1005D0006B817C818E2D0E94E207C70185960E9467
:1005E0006E10682F8E2D0E9404100894E11CF11CDF
:1005F00083E0E816F104B9F62FEF4FEF60E086E1F3
:100600000E948C052FEF4FEF60E086E30E948C057F
:100610002FEF4FEF60E086E50E948C058AE591E0C0
:100620000E946E1080939E048BE591E00E946E10F4
:1006300080939F048CE591E00E946E108093A0044B
:100640008DE591E00E946E108093A1048EE591E00B
:100650000E946E108093A2048FE591E00E946E10BC
:100660008093A30480E691E00E946E1080937C0446
:1006700081E691E00E946E1080937D0482E691E015
:100680000E946E1080937E0483E691E00E946E10BB
:1006900080937F0484E691E00E946E108093800432
:1006A00085E691E00E946E10809381048DEF93E0C7
:1006B0000E946E108093A5048EEF93E00E946E104E
:1006C0008093A6048FEF93E00E946E108093A7049E
:1006D00086E691E00E946E1080934D0187E691E0DE
:1006E0000E946E1080934E0188E691E00E946E1089
:1006F00080934F0189E691E00E946E108093500133
:100700008AE691E00E946E10809351018BE691E0A1
:100710000E946E108093520183E090E00E946E1060
:1007200080FF03C082E08093540183E090E00E9448
:100730006E1082958F70809355010E94512E0E94F9
:10074000AD0378940E9444060E9491110E94DD0A34
:100750000E9440290E94B303F5CF81E080935603A5
:100760001092370408958091BD0481FF07C08091E5
:1007700037048F3F19F08F5F8093370480915603C1
:10078000813051F4809137048F3030F0C09810924E
:10079000370482E08093560380915603823051F4EF
:1007A00080913704853030F0C09A1092370481E090
:1007B000809356030895089508950895089508951F
:1007C00008950895CF92DF92EF92FF920F931F93B7
:1007D000CF93DF93CDB7DEB729970FB6F894DEBF7E
:1007E0000FBECDBF82E00E94B8118CE090E00E9465
:1007F0006E10898382E090E00E946E108A8381E807
:100800008B8381E48C8380915B048D8380915A0477
:100810008E8380915C048F8380915E048887198623
:100820008E010F5F1F4F680189E0E82EF12CEC0E5E
:10083000FD1E8985F8019081890F89878091540177
:10084000882319F480810E94962F0F5F1F4F0E1589
:100850001F0579F780915401882319F489850E9436
:10086000962F80915401882319F0C6010E944534C7
:1008700029960FB6F894DEBF0FBECDBFDF91CF91A2
:100880001F910F91FF90EF90DF90CF900895682F08
:1008900070E080FD2FC0CB018076907035E095959B
:1008A00087953A95E1F7E82FCB018F7990708431E5
:1008B000910529F4F0E0E654FB4F2083089586303B
:1008C000910541F4F0E0EE0FFF1FEC59FB4F208340
:1008D00041830895089771F4F0E0EE0FFF1FEC5488
:1008E000FB4F2083418343FF05C080819181906F3E
:1008F000918380830895EF92FF920F931F93182F97
:10090000062FF42EE22E0E944704C398812F0E94E6
:100910001811802F0E9418118F2D0E9418118E2DF2
:100920000E941811C39A1F910F91FF90EF900895A4
:10093000CF92DF92EF92FF920F931F93CF93DF93AB
:100940007C016B01DC018C9190E09C012F7930706F
:100950002115310519F02830310501F5EC01C0767B
:10096000D07045E0D595C7954A95E1F7C330B0F40E
:100970008C2F8B5E0E94F510682F8C2F0E94041024
:10098000EC2FF0E09F01225B3B4FDF01A05ABF4FED
:100990008C91D9018C93E857FB4F1082F70123818A
:1009A0004281618180810E944704C398C0E0D0E009
:1009B00086010C0F1D1FF701EC0FFD1F80810E94A7
:1009C0001811D8018C932196C430D10589F7C39AA8
:1009D00080E090E0DF91CF911F910F91FF90EF9019
:1009E000DF90CF9008955F926F927F928F929F9247
:1009F000AF92BF92CF92DF92EF92FF920F931F932D
:100A0000CF93DF93CDB7DEB728970FB6F894DEBF4C
:100A10000FBECDBF282F30E0F901E55BFB4F808191
:100A2000882319F4662309F461C060831A82C9011E
:100A3000880F991F820F931F880F991F880F991F86
:100A4000F0E85F2E580E00E010E0862F90E0E4E022
:100A5000AE2EB12CA822B92272E0C72ED12CC8220A
:100A6000D92261E0E62EF12CE822F92255E0652E2C
:100A7000712C6C0E7D1E4E010894811C911CA114DA
:100A8000B10489F0063020F4E114F10421F006C02D
:100A9000C114D10419F490E180E102C091E181E137
:100AA0008B839C830CC0C80185539F4F0E946E109E
:100AB0008B83C80186539F4F0E946E108C83902FAA
:100AC000002311F0063011F480E18C839A3019F480
:100AD0008B8180628B83950D9983B301C4010E9441
:100AE00098040E5F1F4F0C30110549F628960FB67B
:100AF000F894DEBF0FBECDBFDF91CF911F910F9154
:100B0000FF90EF90DF90CF90BF90AF909F908F902D
:100B10007F906F905F9008953F924F925F926F9297
:100B20007F928F929F92AF92BF92CF92DF92EF927D
:100B3000FF920F931F93CF93DF93CDB7DEB7289724
:100B40000FB6F894DEBF0FBECDBFC82E562E442E72
:100B5000322E90E09C012F7930702115310521F063
:100B60002830310509F064C08076907045E0959595
:100B700087954A95E1F7D82E82E08D1508F458C084
:100B8000ED2CFF24F701EE0FFF1FDF01A458BB4F30
:100B90008D919C91EC5BFE4F91838083F701E65B26
:100BA000FE4F8081882371F110821A828CE0D89EDA
:100BB000C00111248C0100581F4F2CE8A22EB12C2B
:100BC000A80EB91E85E0682E712C6C0E7D1E4E019C
:100BD0000894811C911C13C00983C801855B9F4F39
:100BE0000E946E108B83C801865B9F4F0E946E101F
:100BF0008C83B301C4010E9498040E5F1F4F0A1535
:100C00001B0550F38D2D8B5E0E94F510682F8D2DE6
:100C10000E940410D701A25BBB4FF701E05AFF4FBF
:100C200080818C93E8E8F4E0EE0EFF1EF70110825D
:100C3000232D442D652D8C2D0E944704C3988C2DA7
:100C40000E941811852D0E941811842D0E941811E0
:100C5000832D0E941811C39A28960FB6F894DEBF10
:100C60000FBECDBFDF91CF911F910F91FF90EF90FD
:100C7000DF90CF90BF90AF909F908F907F906F90BC
:100C80005F904F903F900895AF92BF92CF92DF92C6
:100C9000EF92FF920F931F93CF93DF93CDB7DEB701
:100CA0002A970FB6F894DEBF0FBECDBF1092400456
:100CB000109241041092420480914904882311F05B
:100CC00083995FC0809114018F5F809314018330FA
:100CD00010F0109214018EE090E00E946E108F5F71
:100CE00080934904809114018295880F807E8B60E7
:100CF0008F838E010D5F1F4F67E0C62ED12CCC0E67
:100D0000DD1EB801C6010E9498048B8180934A04BD
:100D10008D8183FF02C0806F8D838D818A838E8158
:100D20008983E0911401F0E0EE0FFF1FED5BFB4FB4
:100D300089819A8191838083839923C0EE24FF2443
:100D400058011E2D1295110F107E812F87618F8300
:100D5000B501C6010E949804F701E05CFB4F8E814B
:100D6000808316611F838FEF89878A87B501C6014B
:100D70000E9498040894E11CF11C83E0E816F10439
:100D800001F72A960FB6F894DEBF0FBECDBFDF91F4
:100D9000CF911F910F91FF90EF90DF90CF90BF9078
:100DA000AF900895CF93DF93EC0182E090E00E9432
:100DB0006E108093190190911601992359F080913A
:100DC000BD0480FF03C091509093160180911501DE
:100DD00081600EC080911801882339F0809115013F
:100DE00080618093150110921801809115018E7F0A
:100DF0008093150180911801882379F468E0CE0171
:100E00000E944633882349F08F8190911901890F00
:100E10008F8381E08093A40458C00E94722F8F3F7B
:100E200031F4809115018061809315013AC08AE107
:100E300091E00E94B22F8130A1F584E180931601E8
:100E400020911801222329F480911A01809317011F
:100E500025C090911701809119019817D1F4309114
:100E60001501932F94609093150191FD12C0C20F4C
:100E7000D11D219780911A018883283051F494FF65
:100E800004C09F7E9093150106C036603093150113
:100E900002C0283018F01092180103C02F5F209371
:100EA00018011092A4048091150184FF06C08F7E62
:100EB000809315018FEF9FEF0AC081FD03C080E092
:100EC00090E005C08D7F8093150181E090E0DF9177
:100ED000CF910895FB0120813181280F391F35956D
:100EE000279531832083C9010895FF920F931F93A3
:100EF000F62E816080936A040EE614E0B8018AE65B
:100F000094E00E9498040F0D111DF801808190E07B
:100F10001F910F91FF900895816080936A046EE69F
:100F200074E08AE694E00E9498048091710490E055
:100F30000895816080936A046EE674E08AE694E026
:100F40000E9498042091700430E0522F4427809131
:100F5000710490E0482B592B23FD02C0CA0108956B
:100F6000CA01906F0895CF93DF93CDB7DEB7249772
:100F70000FB6F894DEBF0FBECDBF816080936A04C8
:100F80006EE674E08AE694E00E94980490916F0403
:100F900097FF03C08FEF8C8301C01C829B838091DD
:100FA00070048A8380917104898369817A818B813D
:100FB0009C8124960FB6F894DEBF0FBECDBFDF91A3
:100FC000CF910895CF92DF92FF920F931F93CF930B
:100FD000DF93CDB7DEB721970FB6F894DEBF0FBE13
:100FE000CDBF8B01F82EF294FF0C70EEF7228F2DFF
:100FF000896180936A046EE674E08AE694E00E9458
:101000009804C8018070987F892B19F08FEF9FEFAB
:1010100057C080917004982F9F709C5F82958F704D
:10102000981B0F3F1105F9F0F4F06801191694F0C0
:10103000412F5527202F60E08F2D8C600E948C055A
:1010400020E04FE760E08F2D82610E948C0581E0F7
:1010500090E036C0D594C79491508FEFC816D10454
:10106000E1F0DCF0E3CF68019D3094F0412F55278B
:10107000202F60E08F2D8C600E948C052DE040E0D9
:1010800060E08F2D82610E948C0582E090E018C0A4
:10109000CC0CDD1C9F5FC7FEE7CF412F5527202FCB
:1010A00060E08F2D8C6099830E948C059981292F97
:1010B0004C2D60E08F2D82610E948C0580E090E0D5
:1010C00021960FB6F894DEBF0FBECDBFDF91CF9152
:1010D0001F910F91FF90DF90CF9008950F931F9372
:1010E000062F182F1295110F107E812F8561809386
:1010F0006A046EE674E08AE694E00E949804202F69
:101100004091700460E0812F84610E948C051F91E2
:101110000F910895CF93DF93CDB7DEB724970FB625
:10112000F894DEBF0FBECDBF49835A836B837C83A7
:1011300029814A816B810E948C0524960FB6F89410
:10114000DEBF0FBECDBFDF91CF9108951F93182F43
:1011500062E00E946E081295110F107E40E050E090
:1011600060E070E0812F88600E948A0840E050E0D3
:1011700060E070E0812F8A600E948A081F910895C4
:101180008295880F807E40E050E060E070E08860EB
:101190000E948A080895E82FF0E0EE0FFF1FE55146
:1011A000FB4F40815181662329F002C05595479538
:1011B0006A95E2F7509541955F4F662757FD609518
:1011C000762F8295880F807E88600E948A08089515
:1011D000E82FF0E0EE0FFF1FE551FB4F40815181FA
:1011E000662329F002C0559547956A95E2F7662770
:1011F00057FD6095762F8295880F807E88600E94CB
:101200008A0808950F931F93CF93DF93CDB7DEB76E
:1012100022970FB6F894DEBF0FBECDBF8C010197A9
:101220000E946E10FE0131968183C8010E946E10EB
:10123000898389819A8122960FB6F894DEBF0FBE0A
:10124000CDBFDF91CF911F910F910895CF92DF9283
:10125000EF92FF920F931F93CF93DF93CDB7DEB73B
:1012600028970FB6F894DEBF0FBECDBF1A820BECE5
:1012700010E085E0C82ED12CCC0EDD1E7E01089436
:10128000E11CF11C802F8B548983C8010E946E10D1
:101290008B83C80101970E946E108C83B601C70131
:1012A0000E9498040E5F1F4F81E00B34180751F71E
:1012B00028960FB6F894DEBF0FBECDBFDF91CF9159
:1012C0001F910F91FF90EF90DF90CF9008951F93A3
:1012D0009091220180912101981719F480E090E00B
:1012E00040C0E92FF0E0E95CFE4F1081892F8F5F4D
:1012F000809322018A3011F410922201EBEAF4E08B
:10130000119284E0E43BF807D9F78CE090E00E946A
:101310006E108093AB0482E090E00E946E10809388
:10132000AC0480E88093AD048AE88093AE04109307
:10133000B2042091A904233019F4ECEAF4E005C0CA
:101340008091AB048093B304F8CF81919091B30462
:10135000890F8093B30484E0E33BF807B1F7822F51
:1013600090E01F910895EF92FF920F931F938B01CE
:10137000E82EFF24C70125E0880F991F2A95E1F781
:1013800088610E948C07877002C0000F111F8A9528
:10139000E2F7612F772767FD7A95C7014C960E9487
:1013A0007610602FC7014F960E9476101F910F9103
:1013B000FF90EF900895CF92DF92EF92FF920F93FC
:1013C0001F93CF93DF93CDB7DEB728970FB6F8946E
:1013D000DEBF0FBECDBF1A820BE011E035E0C32E99
:1013E000D12CCC0EDD1E7E010894E11CF11C802F57
:1013F0008A548983B601C7010E9498046F81C8018D
:101400000E9476106885C80101970E9476100E5FD1
:101410001F4F81E00B34180751F728960FB6F89448
:10142000DEBF0FBECDBFDF91CF911F910F91FF9017
:10143000EF90DF90CF900895CF92DF92EF92FF92DE
:101440000F931F93CF93DF93CDB7DEB728970FB6D7
:10145000F894DEBF0FBECDBF1A820BEC10E045E062
:10146000C42ED12CCC0EDD1E7E010894E11CF11C93
:10147000802F8A548983B601C7010E9498046F8126
:10148000C8010E9476106885C80101970E947610F5
:101490000E5F1F4F81E00B34180751F728960FB6E7
:1014A000F894DEBF0FBECDBFDF91CF911F910F919A
:1014B000FF90EF90DF90CF9008950F931F93CF93FD
:1014C000DF93082F816007FD24C080936A046EE6D5
:1014D00074E08AE694E00E949804802F0E944010F5
:1014E000CEE6D4E0002711270C1B1D0B080F111DA1
:1014F0006981C8018C0F9D1F0E947610823019F4FB
:1015000082E090E01FC0219684E0C137D80781F7C0
:1015100017C080936A046EE674E08AE694E00E9445
:10152000980410E060917004C801855B9F4F0E9491
:10153000761060917104C801865B9F4F0E947610FF
:1015400080E090E0DF91CF911F910F910895FF927D
:101550000F931F93CF93DF93CDB7DEB728970FB6C6
:10156000F894DEBF0FBECDBFF82E0E944010082FAA
:1015700010E0F982C8010E946E108A83C8010196AA
:101580000E946E108B83C80102960E946E108C839D
:10159000BE016B5F7F4FCE0101960E94980480E0F0
:1015A00090E028960FB6F894DEBF0FBECDBFDF9156
:1015B000CF911F910F91FF9008952F923F924F92DC
:1015C0005F926F927F928F929F92AF92BF92CF92D3
:1015D000DF92EF92FF920F931F93CF93DF9386E0FA
:1015E00090E00E946E10282E809133018F5F8093CF
:1015F00033018150823010F01092330180911B0131
:10160000882369F480E680936A046EE674E08AE6D3
:1016100094E00E94980410921C0181E01BC081306C
:10162000E1F481E680936A046EE674E08AE694E071
:101630000E94980480916E0486FD72C080917004AF
:101640008695809587708093720480917104809351
:101650008B0482E080931B0163C0823009F060C07C
:1016600080911C01A82FB0E0FD01EB55FB4F90814C
:10167000992309F450C0FD01EE58FB4F8081891772
:1016800008F449C015E0AA0FBB1F1A95E1F78A2F8D
:101690008A600E949907BC01892B09F43FC0A09180
:1016A0001C014A2F50E0FA01E654FB4F8081FA01F9
:1016B000EE0FFF1F882319F0EC54FB4F02C0EC59CA
:1016C000FB4F20813181CB0177FF03C0909581953D
:1016D0009F4F37FF03C0309521953F4F82179307E7
:1016E000E9F4FA01EC5CFE4F8081823078F08A2FB9
:1016F0000E94A608E0911C01F0E0DF01A857BB4F53
:1017000081E08C93EC5CFE4F108208C08F5F808379
:1017100010921B0103C0AC5CBE4F1C9210921B01C7
:101720008091BD0480FF3EC20E9407107C0100E052
:1017300010E0E0925104F09252040093530410938D
:1017400054048091550490915604A0915704B0918F
:1017500058048E159F05A007B1078CF5A8019701C5
:10176000281B390B4A0B5B0B2F37310541055105FF
:10177000ACF48091840490918504A0918604B0918A
:101780008704280F391F4A1F5B1F2093840430935E
:101790008504409386045093870443C08091840459
:1017A00090918504A0918604B0918704820F931FC5
:1017B000A41FB51F80509140A040B0402AC0E81639
:1017C000F9060A071B070CF044C09C01AD012E1955
:1017D0003F09400B510B20383105410551054CF4B0
:1017E0008091840490918504A0918604B09187042F
:1017F0000CC08091840490918504A0918604B091DE
:10180000870480509F4FAF4FBF4F821B930BA40B99
:10181000B50B8093840490938504A0938604B093C1
:1018200087048091840490918504A0918604B091EE
:101830008704B0708093840490938504A0938604F9
:10184000B09387048091860487FF03C08FEF809355
:101850008704E0925504F0925604009357041093C5
:10186000580480E00E94F53081E00E94F53082E06B
:101870000E94F5308DE780936A046EE674E08AE694
:1018800094E00E94980410912201E091210170914E
:101890005301A0E0B0E041E050E00A2E02C0440F46
:1018A000551F0A94E2F7642F842F8723D9F0809183
:1018B0006E0490E09D01220F331F02C0959587951D
:1018C0002A95E2F780FF0EC08E2F8F5F8A3009F4D1
:1018D00080E0811729F0F0E0E95CFE4F4083E82FBB
:1018E000609576231196A330B105A9F6E093210106
:1018F000709353018091BD0481FFA7C001E411E002
:10190000EAE46E2EE1E07E2E7DE1872E71E0972ED7
:101910006EE9462E64E0562E5EE4A52E54E0B52E08
:10192000C0E0D0E040E8C42E36E8332ECE0125E0FA
:10193000880F991F2A95E1F78A600E9499077C0118
:10194000F5018081E114F10479F0882341F48C2FB2
:101950008B5E0E94F510682F8C2F0E940410FE01F0
:10196000E05AFF4F80810BC0882341F48C2F0E94E6
:10197000F510682F8C2F0E94041003C08150F501D0
:101980008083F20120813181FFEF2F3F3F07A9F4CF
:10199000F8018081823009F441C021E145E060E036
:1019A0008C2D0E947B0421E14DE060E0832D0E949C
:1019B0007B0482E0F801808331C0C701F7FE03C0D9
:1019C000909581959F4FF80140818217930794F07D
:1019D000413021F127E045E060E08C2D0E947B043E
:1019E0002FE04DE060E0832D0E947B0481E0F80150
:1019F000808310C0442391F020E145E060E08C2D0D
:101A00000E947B0420E14DE060E0832D0E947B0476
:101A1000F8011082F3011082F40110822196FCE09B
:101A2000CF0E3F0E0F5F1F4F0894611C711C08946E
:101A3000811C911C82E090E0480E591E0894A11C64
:101A4000B11C94EAC91609F071CF8CE7482E84E0E6
:101A5000582E0DE1E02E01E0F02E1DE4612E11E084
:101A6000712EBAE48B2EB1E09B2EA4E4CA2EA1E025
:101A7000DA2EAA24BB24FAE83F2EC501E5E0880F40
:101A8000991FEA95E1F78A600E949907EC0197FF98
:101A900003C0D095C195DF4FF20180819181892BE0
:101AA00031F1209721F5F601808191810097D9F4D9
:101AB000F40180818823D9F4132D1A5000E020E12D
:101AC00040E160E0812F0E947B040E5F1E5F0C30BE
:101AD000B1F720E140E360E0832D0E947B0481E0C8
:101AE000F401808304C00197F60191838083AA20CA
:101AF00009F03FC0F30180819181009709F4DEC0B5
:101B0000C817D90708F4DAC0F7018081882309F0E3
:101B1000D5C081E0808300EC10E02CE24CE260E074
:101B2000802F0E947B040E5F1F4FF1E000301F07E3
:101B300009F4C4C0F2CF892BE1F4F7018081882336
:101B4000C1F01082CAE0D1E0CE010E946E10182FC1
:101B5000CE0101960E946E10212F482F60E0FE01F9
:101B6000EA548E2F0E947B042296F1E0CA34DF07EC
:101B700059F70894A11CB11C82E090E0480E591E50
:101B80000894E11CF11C680E791E9CE0390E089443
:101B9000811C911CE2E0F0E0CE0EDF1EFEEA3F1653
:101BA00009F06BCF809159048823F9F484E0809385
:101BB000590468E08EE894E00E948F0FA7B1B0E06E
:101BC000AA0FBB1FAD5DBE4FE7B1F0E0EE0FFF1FE8
:101BD000E257FB4F8D919C91119720813181820FAB
:101BE000931F959587958D939C93809198049091E0
:101BF0009904803F910570F480915601823051F034
:101C000082E08093560181E08093200180E00E9471
:101C1000C008AB9A2091980430919904C901815F62
:101C20009040CB9750F480915601813031F081E0A3
:101C30008093560180932001AB982555314050F098
:101C400080915601882331F01092560181E08093F3
:101C50002001AB9890913301E92FF0E0E758FB4F5A
:101C60008081882319F0892F0E940331222011F1ED
:101C700091E0291619F49A9906C01CC0E2E02E16CC
:101C8000C9F49A9917C0AB9A81E08093A80400E048
:101C900010E062E0802F0E946E08802F0E94C00832
:101CA000F801E758FB4F10820F5F1F4F03301105FB
:101CB00069F0EFCFAB981092A80408C0F3018081BF
:101CC0009181C817D90708F438CF35CFDF91CF916C
:101CD0001F910F91FF90EF90DF90CF90BF90AF904A
:101CE0009F908F907F906F905F904F903F902F903C
:101CF00008951F920F920FB60F9211248F9381E0D7
:101D000080935D048F910F900FBE0F901F901895D8
:101D100010925D0408951F93CF93DF93CDB7DEB784
:101D200022970FB6F894DEBF0FBECDBF23E040E090
:101D300060E084E10E947B0423E040E060E084E313
:101D40000E947B0423E040E060E084E50E947B0485
:101D500020E040E060E08AE00E947B0420E040E078
:101D600060E08AE20E947B0420E040E060E08AE4D8
:101D70000E947B0410E002C01431A1F020E040E09A
:101D800060E0812F0E947B0420E040E060E0812F32
:101D900080620E947B0420E040E060E0812F80644C
:101DA0000E947B041E5F1C3138F320E040E060E0BD
:101DB0008EE70E947B0410E020E040E060E0812F8D
:101DC00080680E947B041E5F1038B1F72FEF47E058
:101DD00060E08AE00E947B041A82198206C000003B
:101DE00089819A8101969A83898389819A81885B06
:101DF0009B40ACF320E040E060E08AE00E947B047E
:101E0000C39883E00E94181180E00E94181180930B
:101E1000610480E00E9418118093600480E00E94B9
:101E2000181180935F04C39A20E040E060E082E0F4
:101E30000E947B0480915F0490916004A0916104F2
:101E4000B0916204805D9740A040B04010F480E102
:101E500001C088E08093630422960FB6F894DEBF39
:101E60000FBECDBFDF91CF911F910895CF93DF9328
:101E7000CDB7DEB722970FB6F894DEBF0FBECDBF49
:101E80008AE08ABB1BBA8FEB87BB8BE188BB8CE0F7
:101E900084BB83EF85BB82EF81BB85E082BBDB988F
:101EA0001A82198206C0000089819A8101969A835C
:101EB000898389819A8184369105ACF31A821982CB
:101EC00006C0000089819A8101969A83898389815D
:101ED0009A8184369105ACF322960FB6F894DEBF52
:101EE0000FBECDBFDF91CF91089581B3806B81BBD1
:101EF00081EA8FBD81E08EBD81E685BD089588238E
:101F000019F41BBC6ABD0895813019F419BC68BD71
:101F1000089563BD089517B886EC86B90895E7B1B2
:101F2000F0E0EE0FFF1FE80FF91F84B195B1918328
:101F3000808387B190E070E061507040861797070A
:101F400024F487B18F5F87B901C017B8369A089516
:101F50000895882311F4D99A0895813009F4DB9A01
:101F60000895882311F4D9980895813009F4DB98F5
:101F70000895882329F489B390E0817090700895C2
:101F8000813019F080E090E0089589B390E0969553
:101F9000879596958795817090700895882331F480
:101FA000662311F0D89A0895D8980895813029F4BD
:101FB000662311F0DA9A0895DA980895882339F49F
:101FC0008BB390E0969587958170907008958130DD
:101FD00019F080E090E008958BB390E043E096958F
:101FE00087954A95E1F781709070089580FF02C04F
:101FF000D99A01C0D99881FF02C0DB9A0895DB9875
:10200000089580E090E008950E947F0F0895CF9397
:10201000DF93CDB7DEB724970FB6F894DEBF0FBEBF
:10202000CDBFC29A8FEF8FB9779BFECF2FB18FEFC5
:102030008FB9779BFECF9FB18FEF8FB9779BFECF84
:102040008FB1C2981C822B839A83898389819A815C
:10205000AB81BC8163E0B695A795979587956A9506
:10206000D1F789839A83AB83BC83898190E02496DE
:102070000FB6F894DEBF0FBECDBFDF91CF910895AC
:10208000282F87FD23C0482F46954F7083E0489F37
:10209000C001112430E0207630702115310511F493
:1020A000CD961AC02032310519F486599F4F14C0BD
:1020B0002034310519F489569F4F0EC04F3019F462
:1020C00087EC90E009C04E3039F404C0265B822FC3
:1020D00090E0089583E090E090E00895DC01E199BC
:1020E000FECF0E940338802D90E008951F93CF9378
:1020F000DF93EC01162F89E090E00E946E10882398
:1021000031F0C930D10519F082E090E008C0E199C2
:10211000FECFDE01012E0E940B3880E090E0DF91BF
:10212000CF911F910895EF92FF921F93CF93DF936A
:102130008DE6E82E80E0F82EC0E1D0E0F7011491A2
:10214000612FCE010E947610612FCE0101960E9470
:102150007610612FCE0102960E9476100894E11C41
:10216000F11C2396CD33D10549F7DF91CF911F9113
:10217000FF90EF900895CF92DF92EF92FF920F932E
:102180001F93CF93DF936C017B01042F10E0C0E01D
:10219000D0E00CC0FE01EE0DFF1DE4916E2FCE01CC
:1021A0008C0D9D1D0E9476101F5F2196101791F7D0
:1021B00080E090E0DF91CF911F910F91FF90EF9021
:1021C000DF90CF900895CF93DF93C0E1D0E0CE01B0
:1021D0000E946E10FE01E95BFE4F80832196CD3395
:1021E000D105A9F7DF91CF910895E7E5F1E0E80F78
:1021F000F11D808190E008958D3218F081E090E02B
:102200000895E82FF0E0E95AFE4F608380E090E007
:10221000089583708DB98DB18C658DB9709A1092C7
:1022200084010895809184011092840190E00895C2
:102230008FB980E009C0893C31F4809184018160CC
:102240008093840103C08F5F779BF5CF769B05C099
:10225000809184018260809384018FB190E0089521
:102260001F920F920FB60F9211248F939F93AF93EB
:10227000BF9380916304883011F482E701C083E248
:1022800082BF8091BE04882319F081508093BE04E0
:1022900080914904882319F08150809349048091EA
:1022A0008801882321F08150809388012BC088E029
:1022B0008093880180918501882319F08150809353
:1022C000850180915904882319F081508093590425
:1022D0008091750490917604A0917704B091780470
:1022E0000196A11DB11D8093750490937604A0936F
:1022F0007704B093780480918204882319F0815088
:1023000080938204BF91AF919F918F910F900FBEE8
:102310000F901F90189582E083BF81E089BF88BF2E
:1023200008951092BD0480918501882301F59AE0FB
:102330009093850181E08093BD048091860188237C
:1023400021F081508093860108959093860183E067
:102350008093BD0480918701882321F08150809370
:10236000870108959093870187E08093BD040895C5
:102370008093B701089599E0699FA001112490E02E
:10238000837090709C01220F331F280F391F420F5A
:10239000531F455E5D4F82E0403D580714F04BE10E
:1023A00052E0CA0108950F931F93CF93DF93CDB7E7
:1023B000DEB728970FB6F894DEBF0FBECDBFE82F6B
:1023C0000D831E832F8338878093FD046093C3049D
:1023D0004093C40481E08093E904388530935B0422
:1023E0002F8120935A049E8190935C048D81809369
:1023F0005E049093AF018093AE013093B3012093BC
:10240000B2019093B1018093B001F0E0EE0FFF1F95
:10241000ED59FF4F0190F081E02D8091E301811192
:10242000099580915B0487FF03C08FEF8C8301C007
:102430001C8280915A048B8380915C048A838091F2
:102440005E04898369817A818B819C8128960FB68D
:10245000F894DEBF0FBECDBFDF91CF911F910F91DA
:1024600008950000089500000895000008950000F8
:1024700008958091C3048823A9F48091D004909199
:10248000D104A091D204B091D3042091B001309135
:10249000B1014091B2015091B301820F931FA41F6B
:1024A000B51FC4C08130A9F48091D0049091D104AB
:1024B000A091D204B091D3042091B0013091B10128
:1024C0004091B2015091B301821B930BA40BB50B49
:1024D000ADC0823099F46091D0047091D1048091A4
:1024E000D2049091D3042091B0013091B101409178
:1024F000B2015091B3010E948B3731C08330D9F4BF
:102500006091D0047091D1048091D2049091D30451
:102510002091B0013091B1014091B2015091B301CD
:102520000E94BE372093D0043093D1044093D2044C
:102530005093D30483C08430D9F46091D004709157
:10254000D1048091D2049091D3042091B0013091B4
:10255000B1014091B2015091B3010E94BE37609326
:10256000D0047093D1048093D2049093D30466C0B6
:102570008530A9F48091D0049091D104A091D20427
:10258000B091D3042091B0013091B1014091B201DA
:102590005091B30182239323A423B52347C08630EF
:1025A000A9F48091D0049091D104A091D204B0916B
:1025B000D3042091B0013091B1014091B20150910A
:1025C000B301822B932BA42BB52B30C08730A9F4F9
:1025D0008091D0049091D104A091D204B091D30401
:1025E0002091B0013091B1014091B2015091B301FD
:1025F00082279327A427B52719C0883069F48091D2
:10260000D0049091D104A091D204B091D3048095CC
:102610009095A095B0950AC0893081F48091B00161
:102620009091B101A091B201B091B3018093D00417
:102630009093D104A093D204B093D3048091D0049A
:102640009091D104A091D204B091D3042091B9010A
:102650003091BA010097A105B10511F4286001C0BD
:10266000277F3093BA012093B90108958091C30464
:102670008823A9F48091D0049091D104A091D20430
:10268000B091D3042091F9043091FA044091FB04F5
:102690005091FC04820F931FA41FB51F16C08130F8
:1026A000E9F48091D0049091D104A091D204B0912A
:1026B000D3042091F9043091FA044091FB04509125
:1026C000FC04821B930BA40BB50B8093D004909356
:1026D000D104A093D204B093D304D8C0823099F42B
:1026E0006091D0047091D1048091D2049091D30470
:1026F0002091F9043091FA044091FB045091FC04BC
:102700000E948B3731C08330D9F46091D00470912E
:10271000D1048091D2049091D3042091F904309196
:10272000FA044091FB045091FC040E94BE372093B0
:10273000D0043093D1044093D2045093D304A6C064
:102740008430D9F46091D0047091D1048091D20486
:102750009091D3042091F9043091FA044091FB0444
:102760005091FC040E94BE376093D0047093D10452
:102770008093D2049093D30489C08530A9F48091CA
:10278000D0049091D104A091D204B091D3042091AF
:10279000F9043091FA044091FB045091FC04822327
:1027A0009323A423B52391CF8630A9F48091D0043C
:1027B0009091D104A091D204B091D3042091F90456
:1027C0003091FA044091FB045091FC04822B932B2E
:1027D000A42BB52B7ACF8730A9F48091D0049091A7
:1027E000D104A091D204B091D3042091F904309186
:1027F000FA044091FB045091FC0482279327A427FC
:10280000B52763CF883069F48091F9049091FA0478
:10281000A091FB04B091FC0480959095A095B09593
:102820000AC0893089F48091D0049091D104A0919C
:10283000D204B091D3048093F9049093FA04A09346
:10284000FB04B093FC0422C08A3001F52091D0042F
:102850003091D1044091D2045091D3048091F90475
:102860009091FA04A091FB04B091FC048093D004F1
:102870009093D104A093D204B093D3042093F9048D
:102880003093FA044093FB045093FC048091D004ED
:102890009091D104A091D204B091D3042091B901B8
:1028A0003091BA010097A105B10511F4286001C06B
:1028B000277F3093BA012093B9010895EF92FF92D8
:1028C0000F931F93E090D004F090D1040091D204B4
:1028D0001091D3042091B0013091B1014091B20127
:1028E0005091B3012E153F05400751073CF48091EC
:1028F000B9019091BA0184608C7F0EC08091B901BA
:102900009091BA01E216F3060407150719F4897FBE
:10291000816002C0887F82609093BA018093B90180
:102920008091B9019091BA01E114F10401051105FA
:1029300011F4886001C0877F9093BA018093B90138
:102940001F910F91FF90EF9008958091C304882309
:1029500039F48091B9019091BA0183FF7AC060C0C7
:10296000813039F48091B9019091BA0183FD71C031
:1029700057C0823029F48091B9019091BA012CC0DE
:10298000833039F48091B9019091BA0180FD61C022
:1029900047C0843039F48091B9019091BA0182FF27
:1029A00058C03EC0853039F48091B9019091BA0188
:1029B00082FD36C011C0863039F48091B901909102
:1029C000BA0181FF46C02CC0873049F48091B9011B
:1029D0009091BA0181FD24C080FF3BC021C08830A6
:1029E00039F48091B9019091BA0184FF32C018C0C6
:1029F000893039F48091B9019091BA0185FF29C0DD
:102A00000FC08A3039F48091B9019091BA0186FFE4
:102A100020C006C08B3069F48091B90187FF19C0CE
:102A20008091AE019091AF019093C1048093C00456
:102A300008958C3071F48091B9019091BA0190FFA2
:102A400008C08091AE019091AF019093C104809332
:102A5000C00408958091AE019091AF019093C1049C
:102A60008093C004089520919A012830B8F4E22F91
:102A7000F0E0EE0FFF1FE657FE4F8091C0049091EB
:102A8000C104918380832F5F20939A018091AE01CE
:102A90009091AF019093C1048093C0040895E09198
:102AA0009A01EE2371F0E150E0939A01F0E0EE0F0D
:102AB000FF1FE657FE4F808191819093C104809360
:102AC000C00408958091C304813011F4809389017A
:102AD00008958091C304813011F410928901089502
:102AE0001092CB0408958091C304882339F4809117
:102AF000B9019091BA018F7090701FC0813031F48C
:102B00008091B9019091BA018F7E17C0823031F463
:102B10008091B9019091BA018F7D0FC0833031F45B
:102B20008091B9019091BA018F7B07C0843051F434
:102B30008091B9019091BA018F779093BA018093F7
:102B4000B9010895853049F48091B9019091BA0195
:102B50009E7F9093BA018093B90108958091C30438
:102B6000813041F480915C048093D60180915E04B1
:102B70008093D701089508950000089500000895F6
:102B800000000895000008950000089500000895D1
:102B900000000895000008950000089500000895C1
:102BA00000000895000008950000089500000895B1
:102BB00000000895000008950000089500000895A1
:102BC0000000089500000895000008950000089591
:102BD0000000089500000895000008951092CB04AD
:102BE00008958091C304813041F48091AE019091A9
:102BF000AF019093C1048093C00481E08093CB0423
:102C0000089582E08093CB04089583E08093CB0401
:102C10001092C1041092C0048FEF9FEF9093BE01F9
:102C20008093BD0110929A011092D40410929B01DE
:102C300081E08093B6011092BC011092BB0110920A
:102C4000D0041092D1041092D2041092D3041092A6
:102C5000890108951092DC041092BC011092BB010E
:102C600008958091C3048130D9F0813030F08230F2
:102C700031F1833009F044C033C08091CB0480939C
:102C80005B048091D40480935A042091BB0130915D
:102C9000BC01832F992780935C0420935E040895E0
:102CA0008091CB0480935B048091D40480935A0478
:102CB0008091C10480935C048091C0040EC0809117
:102CC000D30480935B048091D20480935A04809152
:102CD000D10480935C048091D00480935E040895B5
:102CE0008091FC0480935B048091FB0480935A04E0
:102CF0008091FA0480935C048091F90480935E04CF
:102D0000089580915E048093530181E08093A9042B
:102D10008091A404882319F083E08093A904089586
:102D200080915401882321F481E080935401089517
:102D3000823019F483E08093540108958091C30494
:102D4000813049F08130A0F0823009F44FC08330E7
:102D500009F063C058C04091D4015091D5016091F1
:102D6000AE017091AF01E0ECF1E020E030E03AC05C
:102D70002091D4013091D5012A30310590F4F90128
:102D8000EE0FFF1FE054FE4F8091AE019091AF0116
:102D9000918380832F5F3F4F3093D5012093D401DF
:102DA000089589E08093BF040895819191918617D9
:102DB0009707B1F4F901EE0FFF1FE054FE4F4150A9
:102DC000504006C02F5F3F4F828193818193919342
:102DD00024173507B8F35093D5014093D4010895D3
:102DE0002F5F3F4F2417350701F708951092D50143
:102DF0001092D401E0ECF1E01192119281E0E43DF7
:102E0000F80771F0F9CF10925B0410925A041092F7
:102E10005C048AE080935E04089583E08093BF049D
:102E200008958091F204813881F58091F30482390C
:102E300061F58091F404833A41F58091F504843B77
:102E400021F58091F604853C01F58091F704863DDB
:102E5000E1F4F894C098AB9A89E0E3E0F0E0809365
:102E600057008491867019F40C94003808958230CC
:102E700019F40C94003C0895843019F40C94003E2D
:102E80000895863011F40C94003F0895CF93DF939A
:102E9000CDB7DEB728970FB6F894DEBF0FBECDBF13
:102EA0008091C3048130F1F48091C4048A32C1F46A
:102EB00080915E04898380915C048A8380915A04A6
:102EC0008B8380915B048C831D821E821F821886F7
:102ED000BE016F5F7F4F8FEF97E00E9487302FC05A
:102EE00084E02BC0882341F5BE016F5F7F4F8FEFD9
:102EF00097E00E94573090915E048981981799F469
:102F000090915C048A81981771F490915A048B8196
:102F1000981749F490915B048C81981721F481E013
:102F200080935E0402C010925E0410925B041092C3
:102F30005A0410925C0403C083E08093BF04289677
:102F40000FB6F894DEBF0FBECDBFDF91CF910895CD
:102F50008091CB04882389F1833079F1853069F140
:102F60006CE971E08091C0049091C1040E945730D7
:102F70002091C0043091C1048091BD019091BE01A7
:102F80008217930721F081E08093B60102C010926E
:102F9000B6013093BE012093BD012F5F3F4F3093A8
:102FA000C1042093C0048091CB04823019F485E0E1
:102FB0008093CB0481E090E0089580E090E0089554
:102FC0008CE090E00E946E108093A5018091C30474
:102FD000882399F482E08093B70124E530E0A5EAE4
:102FE000B1E0F9018491FD0181832F5F3F4F11967C
:102FF000F1E0AD3ABF0761F0F4CF10925B0481E0DD
:1030000080935A0483E080935C0485E280935E049D
:1030100008952091AE013091AF013093BC0120930F
:10302000BB0182E08093B7012F5F374078F487E0DF
:1030300090E00E946E1080FD09C066EA71E0809108
:10304000BB019091BC010E94573007C0E5EAF1E056
:10305000119281E0EE3AF807D9F78CE090E00E94F7
:103060006E108093A501089583E08093CB0487E0E0
:1030700090E00E946E1081FD04C081E08093DC042A
:1030800003C088E08093BF048091AE019091AF01AE
:103090009093BC018093BB0108950F931F93CF932E
:1030A000DF93CDB7DEB724970FB6F894DEBF0FBE1F
:1030B000CDBFE82FF0E06623C1F189E0689F800171
:1030C00011249F0123703070C901880F991F820F4E
:1030D000931F080F191F055E1D4F82E00F3C180754
:1030E00044F081E08093BF0460E070E080E090E015
:1030F00026C0C80102960E946E108B83C8010196FB
:103100000E946E10FE0131968183C8010E946E10EC
:1031100089838B8187FF03C08FEF8C8301C01C8262
:1031200069817A818B819C810AC0EE0FFF1FEE0FAF
:10313000FF1FE352FB4F608171818281938124964E
:103140000FB6F894DEBF0FBECDBFDF91CF911F91B8
:103150000F910895CF93DF93CDB7DEB724970FB6C5
:10316000F894DEBF0FBECDBF6091C3048091C4044C
:103170000E944D1869837A838B839C834C81409392
:103180005B043B8130935A042A8120935C0499812B
:1031900090935E048091E9048823F9F04093D3046E
:1031A0003093D2042093D1049093D0048091D00422
:1031B0009091D104A091D204B091D3042091B9018F
:1031C0003091BA010097A105B10511F4286001C042
:1031D000277F3093BA012093B90124960FB6F89453
:1031E000DEBF0FBECDBFDF91CF9108958091AE01BC
:1031F0009091AF01825D944041F460E080E090E006
:103200000E947610F8940C94000008950F931F9379
:10321000CF93DF93CDB7DEB724970FB6F894DEBF18
:103220000FBECDBF9091C304992341F189E0989FCF
:10323000800111248091C40423E0829FC0011124E5
:10324000080F191F055E1D4F82E00F3C180724F080
:1032500081E08093BF0432C060915A04C801029695
:103260000E94761060915C04C80101960E9476105D
:1032700060915E04C8010E94761020C080915A04BB
:103280008B8390915C049A8390915E04998387FF6D
:1032900003C08FEF8C8301C01C82E091C404F0E076
:1032A000EE0FFF1FEE0FFF1FE352FB4F89819A8144
:1032B000AB81BC8180839183A283B38324960FB6B4
:1032C000F894DEBF0FBECDBFDF91CF911F910F915C
:1032D00008959091C30497FF13C08091D304809305
:1032E0005B048091D20480935A048091D10480932E
:1032F0005C048091D00480935E049F779093C30414
:103300008091C304882321F0823011F08330A1F52D
:10331000C39AC49A882311F4AF9807C0823011F47D
:10332000AE9803C0833009F4AD988091C404843012
:1033300030F080915B040E94181180935B048091AF
:10334000C404833030F080915A040E941811809395
:103350005A048091C404823030F080915C040E9451
:10336000181180935C0480915E040E941811809370
:103370005E0485B3806E85BB8091C3048130F1F417
:1033800085B3806E85BBC49AC39880915B040E940C
:10339000181180935B0480915A040E941811809345
:1033A0005A0480915C040E94181180935C048091FF
:1033B0005E040E94181180935E04C39A8091E90410
:1033C000882359F180915B048093D30480915A043F
:1033D0008093D20480915C048093D10480915E0438
:1033E0008093D0048091D0049091D104A091D20414
:1033F000B091D3042091B9013091BA010097A10591
:10340000B10531F428603093BA012093B9010895D1
:10341000277F3093BA012093B90108951F9381E06B
:103420008093D4044091C304442339F08091AE01C9
:103430009091AF011816190604F52091B6012223C8
:1034400041F08091AE019091AF019093B5018093CE
:10345000B401442391F48091AE019091AF018F5F4C
:103460009F4F51F5222341F18091D0049091D104D6
:103470009093B5018093B4011FC08091AE019091EB
:10348000AF01181619061CF020E030E00AC020E059
:103490008091B4019091B501892B09F021E081E080
:1034A0002827122F8091B9019091BA01222311F09F
:1034B000806121C08F7E1FC08091B4019091B501C1
:1034C000892B11F41092D4048091D404882341F004
:1034D0008091BD019091BE019093C1048093C0047E
:1034E0008091B9019091BA018F7E9093BA01809337
:1034F000B90110E025C09093BA018093B901413021
:10350000F9F460E08DE70E94750790E02091C40413
:10351000220F02C0959587952A95E2F780FF02C099
:103520001092D4048091D404882351F0112341F4E3
:103530008091BD019091BE019093C1048093C0041D
:103540008091C304823019F563E08DE70E9475070E
:1035500090E04091C404440F22E030E002C0220F0A
:10356000331F4A95E2F782239323892B11F010929F
:10357000D4048091D404882351F0112341F4809124
:10358000BD019091BE019093C1048093C0048091CD
:10359000C3048330F9F463E08DE70E94750790E07F
:1035A0002091C404220F02C0959587952A95E2F7D1
:1035B00080FF02C01092D4048091D404882351F07B
:1035C000112341F48091BD019091BE019093C104FB
:1035D0008093C0048091C304843009F049C0E09115
:1035E000C404E33050F41092D404F0E0E758FB4FE9
:1035F0008081882379F181E028C0E43049F480910A
:103600007904882301F520E030E080917A0415C028
:10361000E53059F0E63019F48091790408C0E730BC
:10362000B9F480917904882371F480917A04882315
:1036300051F420E030E080917B04882311F021E0F8
:1036400030E0C90102C081E090E08093D40402C060
:103650001092D4048091D404882351F0112341F4B2
:103660008091BD019091BE019093C1048093C004EC
:103670001F9108958091C304882341F4E091C4040C
:10368000F0E0E758FB4F81E080830895813081F4BA
:103690008091C404E82FF0E0E758FB4F9FE090834F
:1036A00062E00E946E088091C4040E94C0080895E0
:1036B000823049F5E091C404F0E0E758FB4FE08127
:1036C000E0935E048091E9048823E9F08E2F90E076
:1036D000A0E0B0E08093D0049093D104A093D204F2
:1036E000B093D3048091B9019091BA01EE2331F4E3
:1036F00088609093BA018093B9010895877F909371
:10370000BA018093B901089562E08091C4040E94D7
:103710006E088091C4040E94C0080895EF92FF9241
:103720000F931F93CF93DF938091C404882341F4B8
:103730008091C304873109F001C10E942609FEC0AF
:10374000813009F0B0C08091C304863038F4C82FAE
:10375000D0E0C759DE4F8330E1F415C0893038F42A
:10376000C82FD0E0CC0FDD1FCC59DE4F12C08C30FB
:1037700008F0E1C0C82FD0E0CC0FDD1FCC0FDD1F5B
:10378000CC5ADE4F06C0CE010E946E1080935203C9
:103790000FC0843031F4CE010E946E10809351032B
:1037A00007C0853029F4CE010E946E108093530328
:1037B0008091C304863061F4CE0101960E946E10A0
:1037C00080935503CE010E946E1080935403B6C0BF
:1037D000873061F4CE0101960E946E1080934E03F3
:1037E000CE010E946E1080934D03A8C0883061F412
:1037F000CE0101960E946E1080935003CE010E946C
:103800006E1080934F039AC08930C1F4CE010396A5
:103810000E946E1080933B04CE0102960E946E10AF
:1038200080933A04CE0101960E946E108093390471
:10383000CE010E946E108093380480C08A30C1F49B
:10384000CE0103960E946E1080933F04CE01029633
:103850000E946E1080933E04CE0101960E946E106D
:1038600080933D04CE010E946E1080933C0466C09C
:103870008B3009F063C0CE0103960E946E108093D6
:103880004C03CE0102960E946E1080934B03CE0132
:1038900001960E946E1080934A03CE010E946E1022
:1038A000809349034BC0823009F048C00091C304A3
:1038B000083308F043C010E0000F111F000F111F64
:1038C000BBE1EB2EB3E0FB2EE00EF11EC7010E9420
:1038D0006E10095A1C4FF80180838091C304C82FD1
:1038E000D0E0CC0FDD1FCC0FDD1FC85ADC4FC70165
:1038F00001960E946E1088838091C304C82FD0E087
:10390000CC0FDD1FCC0FDD1FC75ADC4FC70102965D
:103910000E946E1088838091C304C82FD0E0CC0F22
:10392000DD1FCC0FDD1FC65ADC4FC70103960E9476
:103930006E10888303C0CFEFD3E02BCFDF91CF9100
:103940001F910F91FF90EF9008950F931F93CF93C6
:10395000DF938091C404882321F48091C3048934C7
:1039600049F089E090E00E946E10882319F085E00C
:103970008093BF048091C404882311F58091C3040F
:10398000803428F5873088F4863011F48EE70AC039
:10399000880F880F8C590E945D0A8091C304880F9C
:1039A000880F8A590E945D0AF0C0873019F40E947E
:1039B0001C0AEBC0873109F0E8C00E94DB09E5C0B2
:1039C000813009F09FC08091C304833020F483E0EC
:1039D0008093BF04DAC0863038F4C82FD0E0C759CE
:1039E000DE4F8330C9F415C0893038F4C82FD0E0D9
:1039F000CC0FDD1FCC59DE4F0FC08C3008F0C2C099
:103A0000C82FD0E0CC0FDD1FCC0FDD1FCC5ADE4F0E
:103A100003C06091520309C0843019F460915103CE
:103A200004C0853029F460915303CE010E947610C2
:103A30008091C304863049F460915503CE0101960C
:103A40000E947610609154035BC0873049F4609106
:103A50004E03CE0101960E94761060914D0350C036
:103A6000883049F460915003CE0101960E9476108F
:103A700060914F0345C08930A9F460913B04CE01A9
:103A800003960E94761060913A04CE0102960E943D
:103A9000761060913904CE0101960E9476106091F3
:103AA00038042EC08A30A9F460913F04CE010396F9
:103AB0000E94761060913E04CE0102960E9476101C
:103AC00060913D04CE0101960E94761060913C0405
:103AD00017C08B3009F059C060914C03CE0103969A
:103AE0000E94761060914B03CE0102960E947610E0
:103AF00060914A03CE0101960E94761060914903BD
:103B0000CE013DC0823009F040C0E091C304E833EB
:103B1000E0F5F0E0EE0FFF1FEE0FFF1F8F01055ED7
:103B20001C4FE95AFC4F6381C80103960E9476102E
:103B3000E091C304F0E0EE0FFF1FEE0FFF1FE95A04
:103B4000FC4F6281C80102960E947610E091C30486
:103B5000F0E0EE0FFF1FEE0FFF1FE95AFC4F6181EF
:103B6000C80101960E947610E091C304F0E0EE0FC8
:103B7000FF1FEE0FFF1FE95AFC4F6081C8010E9432
:103B8000761003C0CFEFD3E047CFDF91CF911F91E5
:103B90000F9108950F931F93CF93DF93CDB7DEB7A7
:103BA00028970FB6F894DEBF0FBECDBF8091C40436
:103BB000882309F0DCC08091C30487FD7DC0803478
:103BC00008F041C08630A9F48FE780936A046EE65E
:103BD00074E08AE694E00E949804809171048093D6
:103BE0005E048091700480935C0480916F048093E4
:103BF0005A048091C304873008F449C1880F880FA4
:103C00008B5980936A046EE674E08AE694E00E9421
:103C100098048091710480935E0480917004809375
:103C20005C0480916A048E5F80936A046EE674E09F
:103C30008AE694E00E9498048091710480935A046B
:103C40008091700436C0803519F486E090E008C099
:103C5000813519F487E090E003C090E080549040F3
:103C600010925C040E946E1080935E049091C304D5
:103C7000892F8654823008F00AC1963419F40EE474
:103C800011E002C00AE411E0C8010E946E108093A6
:103C90005E04C80101960E946E1080935C04C80106
:103CA00002960E946E1080935A04C80103960E94E7
:103CB0006E1080935B04EBC010925B0410925A0468
:103CC00010925C04803819F48091CB0416C08138BE
:103CD00019F48091DC0411C0823859F48091C00439
:103CE0009091C104892F992780935C048091C0042E
:103CF00004C0833829F480919B0180935E042FC017
:103D00008438C9F4F8948091750490917604A09158
:103D10007704B091780489839A83AB83BC837894C9
:103D2000898180935E048A8180935C048B81809377
:103D30005A048C8112C0853891F40E9426376D8315
:103D40007E838F8398878D8180935E048E8180939C
:103D50005C048F8180935A04888580935B048091F2
:103D6000C3048F3F09F093C08091B8018EC08130A9
:103D700009F074C010925B0410925A0410925C0413
:103D80008091C304882319F48091560315C08130B3
:103D9000A9F0823019F4809137040EC0833019F4F1
:103DA0008091520309C0843019F48091510304C0FA
:103DB000853021F48091530380935E048091C30485
:103DC000863039F48091550380935C0480915403CC
:103DD0005CC0873039F480914E0380935C048091FD
:103DE0004D0353C0883039F48091500380935C04B4
:103DF00080914F034AC0893079F480913B048093CD
:103E00005B0480913A0480935A0480913904809332
:103E10005C048091380439C08A3079F480913F0481
:103E200080935B0480913E0480935A0480913D040A
:103E300080935C0480913C0428C08B3041F58091D4
:103E40004C0380935B0480914B0380935A048091D0
:103E50004A0380935C048091490317C08230B9F40F
:103E6000E091C304E83398F4F0E0EE0FFF1FEE0F8B
:103E7000FF1FE95AFC4F838180935B04828180930A
:103E80005A04818180935C04808180935E048091D8
:103E9000E904882339F180915B048093D3048091F5
:103EA0005A048093D20480915C048093D104809161
:103EB0005E048093D0048091D0049091D104A091AD
:103EC000D204B091D3042091B9013091BA01009786
:103ED000A105B10511F4286001C0277F3093BA0114
:103EE0002093B90128960FB6F894DEBF0FBECDBF60
:103EF000DF91CF911F910F9108950F931F93CF934F
:103F0000DF938091C404882309F0D9C08091C30451
:103F100087FDA3C0803458F5863061F420915E049B
:103F2000207F60915A046F7C606240915C048EE750
:103F30000E948C050091C304073008F470C110E0A2
:103F4000000F111F000F111F20915E0440915C04AF
:103F500060E0802F8C590E948C0520915A0440917A
:103F60005B0460E0802F8A590E948C0558C1893417
:103F700009F58091AE019091AF0124E0823D920756
:103F800031F410925C0481E080935E040CC0815E89
:103F9000904129F410925C0410925E0404C084E005
:103FA0008093BF043CC160915E0489E090E00E9470
:103FB000761035C1803519F4C6E0D0E015C08135E2
:103FC00029F0C82FD0E0C054D0400EC080915E04CC
:103FD00080FD08C087E090E00E946E1080FF02C064
:103FE0000E94F12FC7E0D0E08091C304873419F418
:103FF000CAE4D1E004C0863411F4CEE4D1E08654A2
:10400000823090F460915B04CE0103960E9476109A
:1040100060915A04CE0102960E94761060915C0471
:10402000CE0101960E94761060915E04CE010E943E
:1040300076108091C304823421F480915E040E9442
:104040003A338091C304833409F0E9C080915E045F
:1040500082958F7080935501E2C0833829F4809156
:104060005E0480939B0121C0843899F4F894809178
:10407000B0019091B101A091B201B091B3018093D0
:10408000750490937604A0937704B09378047894A1
:104090000CC0853851F46091B0017091B1018091EC
:1040A000B2019091B3010E942B378091C3048F3FDE
:1040B00009F0B5C080915E048093B801B0C0813032
:1040C00009F094C08091C304882329F480915E0490
:1040D00080935603A4C0813009F44FC0823029F484
:1040E00080915E04809337049AC0833029F48091D4
:1040F0005E048093520393C0843029F480915E045F
:10410000809351038CC0853029F480915E048093A4
:10411000530385C0863079F480915C0490E0982F39
:10412000882720915E0430E0822B932B90935503D7
:104130008093540374C0873079F480915C0490E0DC
:10414000982F882720915E0430E0822B932B909348
:104150004E0380934D0363C0883079F480915C04F2
:1041600090E0982F882720915E0430E0822B932BDB
:104170009093500380934F0352C0893089F480910B
:10418000B0019091B101A091B201B091B3018093BF
:10419000380490933904A0933A04B0933B043FC091
:1041A0008A3089F48091B0019091B101A091B2015F
:1041B000B091B30180933C0490933D04A0933E04DE
:1041C000B0933F042CC08B3051F58091B001909199
:1041D000B101A091B201B091B301809349039093D2
:1041E0004A03A0934B03B0934C0319C08230B9F437
:1041F000E091C304E83398F4F0E0EE0FFF1FEE0FF8
:10420000FF1FE95AFC4F80915B04838380915A041D
:10421000828380915C04818380915E048083DF913E
:10422000CF911F910F9108953091D30430935B0487
:104230002091D20420935A049091D10490935C046D
:104240008091D00480935E049093AF018093AE017F
:104250003093B3012093B2019093B1018093B001E8
:104260000E947D1F08950F931F93CF93DF93E091DA
:10427000C304E7FD08C0EF3008F0B9C0F0E0E05932
:10428000FE4FE49101C0EF77E093C3049091C30423
:104290009034C8F4E92FF0E00091C4049F3040F45A
:1042A000EE0FFF1F0295000F007E802F8E2B08C09F
:1042B000EB5AFE4F8491880F0295000F007E802BF1
:1042C0000E94A70A94C09B34E1F48091C404C82FD3
:1042D000D0E0CC0FDD1FCE01865A9E4F0E946E109B
:1042E000C256DB4F88838091C404C82FD0E0CC0F26
:1042F000DD1FCE01855A9E4F0E946E10C256DB4FC5
:104300001DC09C34E9F48091C404C82FD0E0CC0FC8
:10431000DD1FCE01805A9E4F0E946E10C458DB4FA5
:1043200088838091C404C82FD0E0CC0FDD1FCE015C
:104330008F599E4F0E946E10C458DB4F898357C01F
:104340009335E1F48091C404C82FD0E0CC0FDD1F79
:10435000CE018A599E4F0E946E10C35BDE4F888348
:104360008091C404C82FD0E0CC0FDD1FCE01895945
:104370009E4F0E946E10C35BDE4FE0CF892F8155A8
:10438000823020F483E08093BF0431C00091C404E4
:104390009D3459F410E0C80183509C4F0E946E1068
:1043A0000B551B4FF801808322C0C02FD0E0C05CAA
:1043B000D04083E0989FC0011124C80FD91FCE01BF
:1043C00040960E946E1080935E04682F8C2F0E948E
:1043D000FC108091C304853451F4CE010D960E94E7
:1043E0006E10682F9E012350822F0E94FC10DF91D7
:1043F000CF911F910F9108951F93CF93DF93E09179
:10440000C304E7FD08C0EF3008F0B3C0F0E0E059A6
:10441000FE4FE49101C0EF77E093C3042091C30401
:104420002034D0F4E22FF0E09091C4042F3040F417
:10443000EE0FFF1F9295990F907E892F8E2B08C04B
:10444000EB5AFE4F8491880F9295990F907E892B9D
:104450000E945D0A182F88C02B34C9F48091C404CF
:1044600090E0880F991FFC01E256FB4F6081865A4D
:104470009E4F0E9476108091C40490E0880F991F8F
:10448000FC01E256FB4F6181855A9E4F1AC02C34C5
:10449000D9F48091C40490E0880F991FFC01E4587E
:1044A000FB4F6081805A9E4F0E9476108091C40419
:1044B00090E0880F991FFC01E458FB4F61818F59F0
:1044C0009E4F0E94761055C02335C9F48091C404D4
:1044D00090E0880F991FFC01E35BFE4F60818A59D1
:1044E0009E4F0E9476108091C40490E0880F991F1F
:1044F000FC01E35BFE4F618189599E4FE2CF2D3471
:1045000051F48091C40490E0FC01EB55FB4F6081B5
:1045100083509C4FD6CF822F8155823010F483E098
:1045200026C08091C404C82FD0E0C05CD04083E096
:10453000289FC0011124C80FD91F8C2F0E94F5108D
:10454000682FCE0140960E947610182F8091C304E8
:10455000853451F49E012350822F0E94F510682F5C
:10456000CE010D960E947610123019F485E08093EA
:10457000BF04DF91CF911F910895DF92EF92FF92D8
:104580000F931F93CF93DF93CDB7DEB724970FB66A
:10459000F894DEBF0FBECDBFE091C304E7FD08C0B5
:1045A000EF3008F00EC2F0E0E059FE4FE49101C098
:1045B000EF77E093C3042091C3042B3108F0B3C01C
:1045C000233041F4E091C404F0E0EE0FFF1FE55109
:1045D000FB4F09C0263061F4E091C404F0E0EE0F17
:1045E000FF1FEB52FB4F818180935C04808190C060
:1045F0009091C404E22FF0E0293058F5EE0FFF1F30
:104600009295990F907E9E2B916090936A046EE62E
:1046100074E08AE694E00E94980480916F0480938D
:104620005A049091700490935C048091710480937B
:104630005E048091C304843008F46CC093FF6AC0A8
:10464000906F90935C048FEF80935A0480935B0487
:1046500061C0EB5AFE4F8491880F9295990F907E1E
:10466000982B916090936A046EE674E08AE694E079
:104670000E9498041C8280916F048B838091700447
:104680008A8380917104898329813A814B815C817D
:10469000E091C3048E2F90E0FC01ED5BFE4FE491AE
:1046A00004C05595479537952795EA95D2F7298304
:1046B0003A834B835C83815D9E4FEE24FF24870108
:1046C00060E070E0FC01D4900FC081E090E0A0E0D9
:1046D000B0E004C0880F991FAA1FBB1FEA95D2F74C
:1046E000E82AF92A0A2B1B2BE62F6F5F7F4FED1567
:1046F00060F3E222F32204231523E982FA820B837A
:104700001C838B8180935A048A8180935C04898105
:1047100080935E0480915A0487FF02C08FEF24C10A
:1047200010925B0423C12E3108F03FC010925B044D
:1047300010925A0410925C0410925E048DE78093EC
:104740006A046EE674E08AE694E00E949804809120
:10475000C3048B3199F48091C404880F22E030E0C7
:1047600002C0220F331F8A95E2F78091710490E016
:1047700028233923232B09F4F9C015C08C3119F4EF
:104780008091710405C08D3109F0F0C080916E04F4
:1047900090E02091C404220F02C0959587952A9538
:1047A000E2F780FFE3C081E09FC0203408F4DEC060
:1047B000203608F09CC01091C404105C83E0289F50
:1047C000C0011124180F253431F4812F83500E9429
:1047D000F51080935C04812F0E94F51080935E0495
:1047E0008091C3048B34A9F4E091C404F0E0EE0F8F
:1047F000FF1FE256FB4F918190935C048081809370
:104800005E0497FF27C08FEF80935B0480935A0468
:1048100021C08C3441F4E091C404F0E0EE0FFF1F9E
:10482000E458FB4F09C0833559F4E091C404F0E02B
:10483000EE0FFF1FE35BFE4F818180935C0407C096
:10484000863541F4E091C404F0E0E05AFF4F8081E6
:1048500080935E048091C3048D3431F4E091C404EC
:10486000F0E0EB55FB4F0FC08E3431F4E091C404FF
:10487000F0E0EE58FB4F07C0803541F4E091C404EE
:10488000F0E0E557FB4F808180935E048091C30484
:104890008135A9F48091840490918504A0918604C7
:1048A000B09187042091CC043091CD044091CE0486
:1048B0005091CF04821B930BA40BB50B07C0873517
:1048C00009F054C00E940710A0E0B0E089839A83E9
:1048D000AB83BC838C8180935B048B8180935A046F
:1048E0008A8180935C04898180935E043FC0223674
:1048F000C1F410925C04E091C404F0E0E853FB4F73
:10490000808181FF04C081E080935E0402C0109228
:104910005E04E091C404F0E0E853FB4F80818D7F9A
:1049200080838091C3048336C1F410925C04E091CB
:10493000C404F0E0E853FB4F808182FF04C081E0B3
:1049400080935E0402C010925E04E091C404F0E023
:10495000E853FB4F80818B7F808380915C0487FFCD
:1049600005C08FEF80935A0480935B048091E90423
:10497000882339F180915B048093D30480915A0499
:104980008093D20480915C048093D10480915E0472
:104990008093D0048091D0049091D104A091D2044E
:1049A000B091D3042091B9013091BA010097A105CB
:1049B000B10511F4286001C0277F3093BA0120931C
:1049C000B90124960FB6F894DEBF0FBECDBFDF91BC
:1049D000CF911F910F91FF90EF90DF9008950F936B
:1049E0001F93CF93DF93982FC82FDD27C7FDD09556
:1049F000FE01EB53FB4F8081882319F480E090E0A7
:104A00001EC010828E01000F111FF801EB52FB4FE8
:104A100060817181892F0E94E20705511B4F25E0BB
:104A2000CC0FDD1F2A95E1F7F8012081418160E07C
:104A3000FE01E6608E2F0E948C0581E090E0DF9100
:104A4000CF911F910F910895CF93DF93CDB7DEB72C
:104A500022970FB6F894DEBF0FBECDBF9091C4046D
:104A6000E92FF0E0EB53FB4F8081813019F4892F5F
:104A70000E94EF248091AE019091AF0190958195B5
:104A80009F4F9A83898362E08091C4040E946E08DC
:104A90008091C4048295880F807E29814A8160E0DC
:104AA00088600E948C058091C4048295880F807E66
:104AB0002FEF47E060E086600E948C05E091C4041F
:104AC000F0E0EB53FB4F82E0808322960FB6F89420
:104AD000DEBF0FBECDBFDF91CF9108959091C4048A
:104AE000E92FF0E0EB53FB4F8081813019F4892FDF
:104AF0000E94EF2462E08091C4040E946E088091BD
:104B0000C4048295880F807E20915E0440915C04ED
:104B100060E088600E948C058091C4048295880FB3
:104B2000807E2FEF47E060E086600E948C05E09178
:104B3000C404F0E0EB53FB4F82E080830895DF92E2
:104B4000EF92FF920F931F93CF93DF93CDB7DEB712
:104B500024970FB6F894DEBF0FBECDBFD62E082F18
:104B600010E0C801E5E0880F991FEA95E1F782603F
:104B70000E94B3079B01AC01DD2069F17801EE0CC6
:104B8000FF1CE00EF11E8BE192E0E80EF91E89E0B9
:104B9000D89EC0011124E80EF91E9FECE91692E0A0
:104BA000F90624F081E08093BF0420C029833A8372
:104BB0004B835C836B81C70102960E947610FE01D5
:104BC00031966181C70101960E9476106981C70103
:104BD0000E9476100BC0000F111F000F111F03520F
:104BE0001B4FF801208331834283538324960FB6F1
:104BF000F894DEBF0FBECDBFDF91CF911F910F9113
:104C0000FF90EF90DF9008951F931091C30480915F
:104C1000C404833010F4612F30C0843041F4612F1C
:104C200080E00E949F25612F81E00E949F25809156
:104C3000C404853041F4612F81E00E949F25612FDB
:104C400082E00E949F258091C404863041F4612F48
:104C500080E00E949F25612F82E00E949F25809125
:104C6000C404873061F4612F80E00E949F25612F8A
:104C700081E00E949F25612F82E00E949F251F9165
:104C80000895CF92DF92EF92FF920F931F93182F08
:104C9000062F8295880F807E82600E94B3076B0189
:104CA0007C01602F812F0E944D186C157D058E05AB
:104CB0009F0529F460E070E080E090E010C0C61627
:104CC000D706E806F9062CF46C197D098E099F09B0
:104CD00006C0C61AD70AE80AF90AC701B6011F9129
:104CE0000F91FF90EF90DF90CF9008950F931F9357
:104CF000182F062F60E00E946E08602F812F0E94FF
:104D00004D18AB01BC01812F8295880F807E0E94D7
:104D10008A081F910F9108954F925F926F927F9230
:104D20008F929F92AF92BF92CF92DF92EF92FF92BB
:104D30000F931F93CF93DF93CDB7DEB728970FB6AE
:104D4000F894DEBF0FBECDBF80915B0488872091B1
:104D50005A042F83F0905C04FE8290915E049D8340
:104D6000E091C304E7FD08C0EF3008F095C1F0E022
:104D7000E059FE4FE49101C0EF77E093C304009146
:104D8000C304003408F0E9C00930C0F58091C404C0
:104D9000063071F46091AE017091AF010E94E2079C
:104DA000E091C404F0E0EE0FFF1FEB52FB4F1FC079
:104DB00020936B04F0926C0490936D04000F829525
:104DC000880F807E802B80936A046EE674E08AE60A
:104DD00094E00E9498048091C304833009F050C18C
:104DE000E091C404F0E0EE0FFF1FE551FB4F80910E
:104DF000AE019091AF019183808342C10031E9F40B
:104E00008091C4048295880F807E816180936A04BA
:104E10006EE674E08AE694E00E9498048091C404EF
:104E20008295880F807E806180936A0490915E04F1
:104E30009F7080916F04807F1FC08091C4040131F6
:104E400069F58295880F807E816180936A046EE6A1
:104E500074E08AE694E00E9498048091C4048295EC
:104E6000880F807E806180936A0490915E049295A1
:104E7000907F80916F048F70982B90936B0480913A
:104E8000700480936C048091710480936D046EE6CD
:104E900074E08AE694E00E949804F2C01C822B839E
:104EA000FA829983E02FF0E0EB5AFE4FE491EE0F87
:104EB000B82EB294BB0C90EEB922BE2A8B2D0E9464
:104EC000B307AB01BC01E091C3048E2F90E0FC015D
:104ED000ED5BFE4FE49101E010E020E030E004C023
:104EE000000F111F221F331FEA95D2F7C980DA8005
:104EF000EB80FC8044245524815D9E4FFC01A490EE
:104F000025C03601470104C095948794779467942F
:104F10008A95D2F7D401C30181709070892B29F052
:104F2000402B512B622B732B0AC0D901C8018095ED
:104F30009095A095B095482359236A237B23000FB1
:104F4000111F221F331F0894411C511C842D4A1429
:104F5000C0F28B2D0E948A0893C00B3441F4E0917B
:104F6000C404F0E0EE0FFF1FE256FB4F13C00C34F9
:104F700041F4E091C404F0E0EE0FFF1FE458FB4F52
:104F800009C0033571F4E091C404F0E0EE0FFF1F97
:104F9000E35BFE4F8091AE019091AF0191838083DE
:104FA00049C0063531F4E091C404F0E0E05AFF4F07
:104FB00007C00D3439F4E091C404F0E0EB55FB4F29
:104FC000908338C00135A1F58C832B83FA829983B5
:104FD0006091840470918504809186049091870487
:104FE00097FF07C090958095709561957F4F8F4F83
:104FF0009F4F2FEF30E040E050E00E94BE376093BB
:10500000CC047093CD048093CE049093CF04298177
:105010003A814B815C81260F371F481F591F20930F
:10502000840430938504409386045093870402C01F
:10503000003630F51091C404105C83E0089FC00175
:105040001124180F053429F46F2D812F83500E94ED
:10505000FC1060915E04812F0E94FC108091C404BA
:105060008B5E0E94F510682F8091C4040E9404108A
:105070008091C304873411F0803411F410925C04E1
:10508000888580935B048F8180935A048E818093FE
:105090005C048D8180935E0428960FB6F894DEBF81
:1050A0000FBECDBFDF91CF911F910F91FF90EF9079
:1050B000DF90CF90BF90AF909F908F907F906F9038
:1050C0005F904F9008953091D30430935B0420910A
:1050D000D20420935A049091D10490935C0480915F
:1050E000D00480935E049093AF018093AE0130931F
:1050F000B3012093B2019093B1018093B0010E945B
:105100008C26089510925B0410925A0410925C044D
:105110008091C404882331F58091C304883018F449
:105120000E94B90F1DC08A30A0F40E94011090E0C7
:105130002091C30430E02850304002C095958795F7
:105140002A95E2F780FF02C081E00AC010925E0457
:1051500009C083B390E09695879596958795817061
:1051600080935E048091C404813081F4E091C30493
:10517000F0E0EE0FFF1FE257FB4F2081318181816C
:10518000837080935C0420935E0408C0823031F405
:105190008091C3040E94DE0F80935E048091E90435
:1051A000882359F180915B048093D30480915A0441
:1051B0008093D20480915C048093D10480915E043A
:1051C0008093D0048091D0049091D104A091D20416
:1051D000B091D3042091B9013091BA010097A10593
:1051E000B10531F428603093BA012093B9010895D4
:1051F000277F3093BA012093B90108958091C404A8
:10520000882339F460915E048091C3040E94CE0F1C
:105210000895823071F480915E0480FF05C0809112
:10522000C3040E94A90F08958091C3040E94B10F86
:1052300008958F3F21F560915E0480E00E94F304A1
:1052400060915C0481E00E94F30460915A0482E062
:105250000E94F30480915E0482FF03C080E00E94FC
:10526000C00880915C0482FF03C081E00E94C008F6
:1052700080915A0482FF03C082E00E94C008089512
:105280001F93CF93DF938091C80490914004892BA2
:105290008093C8048091C90490914104892B809324
:1052A000C904809142049091CA04892B8093CA0456
:1052B0008091A804882349F08091B9019091BA01A6
:1052C00091609093BA018093B9018091BD0480FFF1
:1052D0000BC08091B4019091B501009729F001971E
:1052E0009093B5018093B4010E946709982F809331
:1052F000E2012091E0013091E1012130310519F006
:10530000882309F459C08091A404882319F49330A8
:1053100091F406C0933021F068E086EA91E003C082
:1053200068E08CEA94E00E9464338091E0019091FF
:10533000E1018E7F48C280918204882309F047C230
:1053400080915401913029F12E7F3093E101209317
:10535000E001823090F4C5EAD1E089910E94962F55
:1053600021E0CE3AD207C9F780915401813009F08B
:105370002EC282E0809354012AC285EA91E00E9405
:10538000453480915401833009F021C210925401B8
:105390001EC2882351F4CBEAD4E089910E94962F53
:1053A00084E0C43BD80729F0F8CF85EA91E00E9459
:1053B00045341092E2010BC21092BF01809154015A
:1053C000882331F481EF94E00E94D206813051F0BD
:1053D000809154018823A1F181EF94E00E94DB3495
:1053E000813071F581E08093BF018091F104809359
:1053F000FD048091F2048093C3048091F3048093B0
:10540000C4048091F40480935B048091F50480933C
:105410005A048091F60480935C048091F704809391
:105420005E048091CB04882319F481E090E053C09E
:1054300020E030E0833011F421E030E0C9014BC0BE
:105440008091BD0482FF23C08091CB04813009F09C
:1054500044C090918901913009F03FC083E080936E
:10546000BF0187E18093FD041092C3041092C4042D
:1054700010925B0410925A048091D60180935C04D0
:105480008091D70180935E049093E90426C00E9426
:10549000A817882311F182E08093BF0180919C01BD
:1054A0008093FD0480919D018093C30480919E01AF
:1054B0008093C40480919F0180935B048091A0013C
:1054C00080935A048091A10180935C048091A20191
:1054D00080935E0481E08093E9048091BF0188237A
:1054E00009F475C182E090E00E946E10382F80931D
:1054F000DB0420915C042093AF0190915E049093B3
:10550000AE0180915B048093B30180915A04809333
:10551000B2012093B1019093B0011092BF04909119
:10552000FD04892F8854883310F09E3870F08091E4
:10553000BF01813011F4923F41F082E08093BF04BB
:1055400080919B01816080939B018091BF0181309C
:1055500091F4E1EFF4E08191380F24E0E83FF207A5
:10556000D1F73093DB048091F8043817C9F081E05B
:105570008093BF0415C0823099F4ECE9F1E0819189
:10558000380F81E0E33AF807D1F73093DB048091DC
:10559000A301381729F080919B01826080939B01C1
:1055A0001092B7018091BF04882309F095C08091C3
:1055B000DC04882311F097FF50C0923F21F40E9431
:1055C000111782E087C0E92FF0E097FF05C0EE0FCA
:1055D000FF1FED50F04004C0EE0FFF1FED59FF4FCD
:1055E0000190F081E02D84E68093BF048091E30177
:1055F000882311F0099503C08FEF8093BF04609159
:10560000D4017091D5016115710509F465C08091CF
:10561000CB04813009F060C08091BF01823009F075
:105620005BC04091C0045091C10420E030E00FC045
:105630002F5F3F4FEE0FFF1FE054FE4F808191819F
:105640004817590721F485E08093CB0445C0E22F29
:10565000F0E0E617F70760F33FC08091BB0190913F
:10566000BC0127E08F3F9207A0F561EF74E00E9434
:105670008730882371F568ED71E08091BB019091CE
:10568000BC010E94573085E68093BF0420E030E0E3
:10569000F901E852FE4FD901AF50BB4F90818C9178
:1056A000981721F087E08093BF0405C02F5F3F4F1C
:1056B0002830310569F78091BF04853669F48091FF
:1056C000BB019091BC0101969093BC018093BB01FA
:1056D00003C087E08093BF048091BF01813009F04F
:1056E00076C08CE090E00E946E10182F82E090E06F
:1056F0000E946E10282F8093C2048091B7018823E6
:10570000C9F59091FD04963031F480915A04880FC8
:10571000880B80935B041093A5012093A6018091D0
:10572000BF048093A7019093A80180915B048093AC
:10573000A90180915A048093AA0180915C0480930E
:10574000AB0180915E048093AC018091A404882316
:1057500039F01092DB049091DB04E6EAF1E003C03B
:105760001093DB04F8CF8191980F81E0ED3AF807B0
:10577000D1F70FC0813089F41093A5011092DB049A
:10578000E5EAF1E090E08191980F21E0ED3AF2072F
:10579000D1F79093DB049093AD018BE090E00E94F1
:1057A0006E10809382048091B801882351F080911B
:1057B000FD04863031F08A3021F08F3011F08F31C6
:1057C00031F481E090E09093E1018093E001DF917A
:1057D000CF911F9108959F92AF92BF92CF92DF9287
:1057E000EF92FF920F931F93CF93DF93CDB7DEB766
:1057F00022970FB6F894DEBF0FBECDBF6C017B01C0
:10580000042F6115710509F499C0009709F496C039
:105810006817790709F492C0142F1295110F107EA2
:10582000A6E09A2E912A892D0E9499079A8389834E
:10583000812F8C600E9499075C0180E0D7FC07C033
:10584000EE0CFF1CCC0CDD1C8F5F8F30B9F7E11420
:10585000F10419F471E0E72EF12C40E050E001C0B2
:105860007901142F4F5F5F4FC70180709E7F9701B2
:1058700036952795892BA1F7C9018C0D9D1DB70180
:105880000E94AA37FB01672B11F4E1E0F0E0898167
:105890009A8154E0880F991F5A95E1F7BF010E9441
:1058A000AA379B01C50144E0880F991F4A95E1F78B
:1058B000BF010E94AA37412F50E0153090F484E0D8
:1058C00090E0841B950B082E02C0369527950A940C
:1058D000E2F73A83298302C0769567958A95E2F7C5
:1058E0000FC0CA010497082E02C0220F331F0A946A
:1058F000E2F73A83298302C0660F771F8A95E2F7A1
:1059000089819A81892B21F481E090E09A838983AF
:105910006115710511F461E070E0749718F4802F3F
:105920000E94E20729814A8160E0892D0E948C054E
:10593000E02FF0E0EB53FB4F81E0808322960FB61F
:10594000F894DEBF0FBECDBFDF91CF911F910F91B5
:10595000FF90EF90DF90CF90BF90AF909F90089511
:105960000F931F93CF93DF93CDB7DEB762970FB638
:10597000F894DEBF0FBECDBF082F162F8430C1F4C0
:1059800080E00E94EF2481E00E94EF24612F80E0FC
:105990000E9441266F83788789879A87612F81E0EB
:1059A0000E9441266B877C878D879E87198A3FC01E
:1059B000853041F481E00E94EF2482E00E94EF24D0
:1059C000198625C0863081F480E00E94EF2482E0B1
:1059D0000E94EF24612F80E00E9441266F83788728
:1059E00089879A871D861BC0873009F580E00E9451
:1059F000EF2481E00E94EF2482E00E94EF24612FD7
:105A000080E00E9441266F83788789879A87612F7B
:105A100081E00E9441266B877C878D879E87612F5E
:105A200082E00E9441266F87788B898B9A8B9985BB
:105A3000992331F48D85882319F48989882369F0A5
:105A40009A83FE013796818189838D858C838C852D
:105A50008B8389898E8388890BC088858A838F810F
:105A600089838C858C838B858B8388898E838F85B6
:105A70008D83043049F429813A818B819C8182177E
:105A80009307D0F441E015C0053049F42B813C81E7
:105A90008D819E818217930758F041E00EC0063039
:105AA00071F429813A818D819E818217930720F4B8
:105AB00042E0BC01C90133C040E0B90130C0073049
:105AC00081F589819A812B813C81ED81FE812817A6
:105AD000390768F4E817F907C0F441E0B9010E94FA
:105AE000EB2B6D817E8142E089819A8118C0E2179B
:105AF000F30758F440E0BC01C9010E94EB2B6D8113
:105B00007E8142E08B819C810AC040E0BC01CF01D4
:105B10000E94EB2B6B817C8141E08D819E810E94F4
:105B2000EB2B62960FB6F894DEBF0FBECDBFDF91B0
:105B3000CF911F910F910895CF92DF92EF92FF9234
:105B40000F931F93CF93DF93CDB7DEB724970FB694
:105B5000F894DEBF0FBECDBF8091C304823008F041
:105B60004BC060E08091C4040E946E088091C40420
:105B70000E94EF246E010894C11CD11C80915B042B
:105B80008C8380915A048B8380915C04F60181831D
:105B900080915E0489838091C304813009F5E98096
:105BA000FA800B811C818091C4048295880F807ECD
:105BB00082600E94B307E60EF71E081F191FE982D4
:105BC000FA820B831C838C8180935B048B8180938E
:105BD0005A04F601818180935C04898180935E047C
:105BE00049815A816B817C818091C4048295880FA0
:105BF000807E0E948A0846C0823009F043C0E0904F
:105C00005E048091C404833030F40E94EF246E2D32
:105C10008091C40435C06E2D0E94B02C8091C404C4
:105C2000843041F46E2D80E00E9476266E2D81E056
:105C30000E9476268091C404853041F46E2D81E067
:105C40000E9476266E2D82E00E9476268091C40402
:105C5000863041F46E2D80E00E9476266E2D82E023
:105C60000E9476268091C404873061F46E2D80E016
:105C70000E9476266E2D81E00E9476266E2D82E0AF
:105C80000E94762624960FB6F894DEBF0FBECDBFD5
:105C9000DF91CF911F910F91FF90EF90DF90CF9008
:105CA0000895CF92DF92EF92FF920F931F93CF93BD
:105CB000DF931092C1041092C0048FEF9FEF909376
:105CC000BE018093BD018DE090E00E946E10813096
:105CD00011F48093CB0415EDC12E14E0D12EBBEE50
:105CE000EB2EB4E0FB2EC0E0D0E0CE018295880F11
:105CF000807E182F8C600E949907F6018193919302
:105D00006F01812F86600E949907F701819391931B
:105D10007F012196C330D10541F707E513E0CEE1BD
:105D2000D3E0CE010E946E10F8018383CE0101976B
:105D30000E946E10F8018283CE0102970E946E10BD
:105D4000F8018183CE0103970E946E10F8018083D1
:105D500024960C5F1F4FF3E0CE3FDF0711F7ECEF07
:105D6000FFE7E491E73299F4EDEFFFE7E491E831E2
:105D700071F4EEEFFFE7E491E83249F4EFEFFFE76B
:105D8000E491E83121F481E08093E30102C01092B4
:105D9000E301DF91CF911F910F91FF90EF90DF9082
:105DA000CF9008951F920F920FB60F9211248F93E8
:105DB0009F93EF93FF938BB1887129F08091E40159
:105DC00080628093E401869B04C08CB180931602AC
:105DD0001AC0809100029CB1E82FF0E0EB51FE4F19
:105DE00090838F5F809300028B3110F0109200023D
:105DF0009091000280910102981729F48091E401AA
:105E000080688093E401FF91EF919F918F910F90B3
:105E10000FBE0F901F9018951F920F920FB60F9202
:105E200011248F939F93EF93FF939091150280918C
:105E30001402981781F0969AE92FF0E0EE5FFD4F7B
:105E400080818CB9892F8F5F80931502823120F079
:105E50001092150201C05598FF91EF919F918F917B
:105E60000F900FBE0F901F9018951F920F920FB6B4
:105E70000F9211248F939F93909115028091140299
:105E8000981709F496989F918F910F900FBE0F90DD
:105E90001F901895982F80910002809301028091A5
:105EA0001502809314021092E401209163042830BB
:105EB00019F4EEE7F1E002C0E7E8F1E0849189B976
:105EC00088ED8AB9992369F0993058F4E92FF0E008
:105ED000283019F4E258FE4F02C0E957FE4F849172
:105EE00089B908958091E40181FF02C01092E40114
:105EF0008BB1887129F08091E40180628093E40184
:105F00008091E40182608093E401807F19F08FEF3B
:105F10009FEF089520E030E090910102809100020F
:105F2000981711F021E030E0C9010895969A9091F8
:105F30001402E92FF0E0EE5FFD4F80839F5F9093A6
:105F40001402923110F01092140290911402809178
:105F50001502981729F48091E40180648093E4018C
:105F6000559A0895DC0190910102809100029817E2
:105F700019F480E090E00895E92FF0E0EB51FE4F36
:105F800080818C93892F8F5F809301028B3118F46D
:105F900081E090E008951092010281E090E0089580
:105FA000209114022E5F30911502223138F080E0EA
:105FB00090E0332349F481E090E0089580E090E0A0
:105FC000231711F481E090E0089520E030E09091F3
:105FD000150280911402981711F421E030E0C901F4
:105FE0000895EF92FF920F931F93CF93DF93CDB756
:105FF000DEB722970FB6F894DEBF0FBECDBF1A8270
:1060000019827E010894E11CF11C34C0C49886E01A
:106010000E941811C49AC49882E00E941811F701D6
:1060200081810E94181189810E94181100E010E0FE
:1060300089819A81800F911F885F9F4340F480E09F
:106040000E9418110F5F1F4F0034110589F7C49A81
:1060500000E010E015C0C49A07C0C49A0F5F1F4F3C
:106060002EE2003E120761F489819A81805C9F4F85
:106070009A83898389819A818050904438F20AC03A
:10608000C49885E00E94181180E00E94181180FDDC
:10609000E4CFE1CF22960FB6F894DEBF0FBECDBF9E
:1060A000DF91CF911F910F91FF90EF900895EF92A4
:1060B000FF920F931F93CF93DF937B018C0193E0AB
:1060C000000F111F9A95E1F7C49883E00E94181100
:1060D000812F99270E941811802F0E941811C0E06B
:1060E000D0E087010C0F1D1F80E00E941811F801FD
:1060F00080832196C830D105A1F7C49A80E090E052
:10610000DF91CF911F910F91FF90EF900895EF9243
:10611000FF920F931F93CF93DF937B018C0133E0AA
:10612000000F111F3A95E1F7C49886E00E941811FC
:10613000C49AC49882E00E941811812F99270E9466
:106140001811802F0E941811C0E0D0E0F701EC0F69
:10615000FD1F80810E9418112196C830D105B1F72A
:10616000C49AC0E0D0E00DC0C49A80E090E013C0B3
:10617000C49A21968EE2C03ED80719F48FEF9FEFA4
:106180000AC0C49885E00E94181180E00E9418118E
:1061900080FDEECFE9CFDF91CF911F910F91FF905E
:1061A000EF90089590917104969590937104809169
:1061B000700480FF03C09068909371049091700404
:1061C00096959093700480916F0480FF03C090684F
:1061D0009093700480916F04869580936F0486FF7E
:1061E00003C0806880936F040895E82FF0E0EE0FFD
:1061F000FF1FE85DFD4F80819181009719F00197A5
:10620000918380830895BF92CF92DF92EF92FF92A5
:106210000F931F93CF93DF93082FC82EDD24F60131
:10622000E758FB4F108123E0B22EB80E8B2D0E9451
:10623000F510E601CC0FDD1F843098F48DE70E9445
:106240008C0722E030E00C2E02C0220F331F0A948C
:10625000E2F7F82EF2228DE70E948C0721E030E071
:1062600012C08DE70E948C0721E030E00C2E02C0A6
:10627000220F331F0A94E2F7F82EF2228DE70E94D4
:106280008C0722E030E002C0220F331FCA95E2F7EC
:106290008223E02EE294EE0CB0EEEB22113019F5E1
:1062A000F601EE0FFF1FE85DFD4F1182108285E1C0
:1062B000E82AE0926A046EE674E08AE694E00E94BE
:1062C0009804F601EB5DFD4F80917004808362E0DD
:1062D000802F0E946E088B2D0E94F510823008F4EA
:1062E000B8C112E0B7C1123051F4802F8A5F0E940A
:1062F000F510682F802F0E94E80813E0ABC113301F
:1063000021F4882309F0A5C1A5C1143051F4802FD0
:106310008A5F0E94F510682F802F0E94CB0815E03D
:1063200099C1153089F4FF2009F494C1802F0E948F
:10633000C008F601EE0FFF1FE85DFD4F8EE190E013
:106340009183808316E086C11630A1F4F601EE0F2A
:10635000FF1FE85DFD4F80819181892B09F07AC193
:10636000802F875F0E94F510682F802F0E94E80819
:1063700017E070C11730D9F4FF2009F06BC122E09B
:1063800043E060E08E2D84610E948C0520E040E0B7
:1063900060E08E2D8C610E948C05802F875F0E94AB
:1063A000F510682F802F0E94CB0818E053C11830D9
:1063B00011F5FF2009F44EC1802F0E94C0088E2DD8
:1063C0008D6180936A046EE674E08AE694E00E9430
:1063D0009804209171044091700460916F048E2D97
:1063E0000E948C0520E043E060E08E2D84610E94D5
:1063F0008C0519E02FC1193009F041C08DE7809359
:106400006A046EE674E08AE694E00E949804809143
:106410006E0490E09601220F331F02C09595879578
:106420002A95E2F780FF16C18B2D0E94F510182FD8
:1064300062E0802F0E946E08802F0E94C00820E03A
:1064400040E060E08E2D0E948C0520E040E060E09E
:106450008E2D82600E948C05133039F080911702D6
:1064600090911802892B09F473C0802F875F0E94D6
:10647000F510682F802F0E94CB081AE0EBC01A306D
:1064800061F4FF2009F4E6C020E040E060E08E2DDA
:106490008C610E948C051BE0DDC01B3009F05AC0E6
:1064A000FF2009F0D7C0802F0E94C0088E2D8D617B
:1064B00080936A046EE674E08AE694E00E94980491
:1064C0000E94D230209171044091700460916F0459
:1064D0008E2D0E948C0520E043E060E08E2D8461CB
:1064E0000E948C0510917104109510937104009115
:1064F0007004009500937004F0906F04F094F09293
:106500006F040E94D23080917104810F80937104D6
:10651000882329F4809170048F5F809370048091A8
:106520007004800F80937004882329F480916F0495
:106530008F5F80936F0460916F046F0D60936F04A1
:1065400020917104409170048E2D8A610E948C0507
:106550001EE080C01E3009F06EC080916E0490E095
:106560009601220F331F02C0959587952A95E2F771
:1065700080FF70C062E0802F0E946E08802F0E9412
:10658000C0088B2D0E94F510833031F080911702E6
:1065900090911802892B91F010926E0410926F0462
:1065A00010927004F601EE0FFF1FEE0FFF1FE75E63
:1065B000FD4F108211821282138203C08E2D0E9421
:1065C000A70A209171044091700460916F048E2D90
:1065D0000E948C051E2D1260209171044091700460
:1065E00060916F04812F0E948C0520E040E060E004
:1065F0008E2D0E948C0520E040E060E0812F0E94FB
:106600008C05F601EB5DFD4F20E0408160E08E2DB2
:1066100084610E948C05F601EE0FFF1FE551FB4FD0
:1066200040815181662757FD6095762F8E2D8660BB
:106630000E948A080CC01F3069F4F601EB5DFD4F23
:1066400022E0408160E08E2D84610E948C0510E084
:1066500001C014E0E9E7F4E0CE0EDF1EF60110837E
:10666000DF91CF911F910F91FF90EF90DF90CF902E
:10667000BF900895823010F482E001C08E7F82B90D
:1066800085EC86BF85B3836085BB0895DC0190915E
:106690002E02961719F080E090E0089540E020E087
:1066A00030E00BC0F901EF5CFD4F8081FD01E20F8E
:1066B000F31F80834F5F2F5F3F4F491799F7109269
:1066C0002E0281E090E00895DC0140E020E030E01F
:1066D0000BC0FD01E20FF31F8081F901E65CFD4F65
:1066E00080834F5F2F5F3F4F461799F760933002CB
:1066F00008951F920F920FB60F9211248F939F93BC
:10670000EF93FF9381B1803629F485EC86BF109218
:106710002E0253C081B1803819F081B1883871F4EC
:1067200085EC86BF80912E02E82FF0E093B1EF5CFC
:10673000FD4F90838F5F80932E023FC081B1803ADE
:10674000D1F181B1882311F485ED36C081B1883A49
:10675000B1F410922F0290912F02E92FF0E0E65C45
:10676000FD4F808183B99F5F90932F0285EC86BF98
:1067700090912F02809130029817F9F416C081B1E0
:10678000883BC9F490912F02E92FF0E0E65CFD4FC1
:10679000808183B99F5F90932F0285EC86BF909193
:1067A0002F0280913002981741F480912F0281507E
:1067B00080932F0202C085EC86BFFF91EF919F91DD
:1067C0008F910F900FBE0F901F90189580914702E8
:1067D00090914802FC0105C02C3211F4108204C0D3
:1067E000319620812223C1F73196F0934802E0933D
:1067F00047020895CF92DF92EF92FF920F931F937B
:10680000CF93DF93CDB7DEB764970FB6F894DEBFB2
:106810000FBECDBF6B017C010E94E52F8823E1F301
:1068200080E20E94962F2AE030E08E010F5F1F4F1A
:10683000A801C701B6010E944737EE24FF24680172
:106840000DC00E94D02F8823E1F70C0D1D1DF8010B
:1068500080810E94962F0894E11CF11C0E2D10E0FF
:10686000F601E00FF11F8081882359F764960FB677
:10687000F894DEBF0FBECDBFDF91CF911F910F9176
:10688000FF90EF90DF90CF9008950F931F93CF93D9
:10689000DF93CDB7DEB724970FB6F894DEBF0FBEF7
:1068A000CDBF8C010E94E52F8823E1F3F8018081A0
:1068B000805C0E94962FF8018181805C0E94962F57
:1068C000F801628170E080E090E00E94FA33F80104
:1068D00084818C8385818B8386818A838781898368
:1068E00069817A818B819C810E94FA338DE00E94BC
:1068F000962F24960FB6F894DEBF0FBECDBFDF9162
:10690000CF911F910F910895CF92DF92EF92FF9256
:106910000F931F93CF93DF93EC0101C02196188151
:10692000812F90E00E94FB37892BC1F71D3229F49B
:10693000219681E0C82ED12C05C01B3209F4219686
:10694000CC24DD2420E030E040E050E01AC0FF24F9
:1069500000E010E080ED9FEFAFEFBFEFE80EF91E13
:106960000A1F1B1FCA01B9012AE030E040E050E0D5
:106970000E948B379B01AC012E0D3F1D401F511F04
:106980002196E8808E2D90E0C0970A9700F3CD28DD
:1069900039F050954095309521953F4F4F4F5F4FBF
:1069A000CA01B901DF91CF911F910F91FF90EF9034
:1069B000DF90CF9008958F929F92AF92BF92CF9227
:1069C000DF92EF92FF920F931F93CF93DF93CDB798
:1069D000DEB725970FB6F894DEBF0FBECDBF5C01C2
:1069E000CE0101960E94B22F882309F4FAC080914B
:1069F00044028823A9F5098110E082E090E00E941A
:106A00006E1090E0805C9F4F0817190789F4809101
:106A1000450290914602892B09F0E3C081E0809302
:106A2000440280915501882309F0DBC08981D7C0D9
:106A300089818D3011F08B3129F410924602109229
:106A40004502CFC080914502909146028F37910553
:106A500008F0C7C001969093460280934502C1C0DA
:106A600080915501882319F489810E94962F2981EC
:106A7000203268F080914502909146028F3791054F
:106A8000A8F4FC01E75BFD4F208301960AC0283083
:106A900069F48091450290914602009709F491C0F3
:106AA000019790934602809345028BC02D3009F0E8
:106AB00088C08091450290914602892B09F481C0DB
:106AC00080915501813021F50E94E52F8823E1F363
:106AD00082E090E00E946E10805C0E94962F00E0A1
:106AE00010E00CC00E94D02F8823E1F7F801E75B8B
:106AF000FD4F80810E94962F0F5F1F4F80914502AE
:106B0000909146020817190768F38DE00E94962FAE
:106B1000109248031092470320914502309146029B
:106B2000609147027091480249E452E090E0A0E091
:106B3000B0E0240F351F2EC0913081F0913018F055
:106B4000923031F51CC0FA018081803209F1FD01DB
:106B5000E853FD4F8083119691E01AC0FA018081BD
:106B6000803289F4A230B10528F0FD01E853FD4FD1
:106B700010821196BD0168537D4F92E009C0FA0161
:106B80008081803229F0FD01E853FD4F808311960A
:106B90004F5F5F4F4217530779F670934802609337
:106BA0004702B0934803A0934703A853BD4F1C92DC
:106BB00081E08093430210924402109246021092A8
:106BC000450289818B3169F4109246021092450288
:106BD0001092440280915501882319F48DE00E949F
:106BE000962F80914302882319F480E090E0BCC086
:106BF00010924302CC24DD2428EC822E22E0922E37
:106C0000760193E0EE0CFF1C9A95E1F7EC18FD0875
:106C1000870100571E4FB801C4010E943437892BE9
:106C200061F4F701EB56FE4F8491F701EA56FE4FEF
:106C3000E491982F3E2F21E00EC0F8018491882323
:106C400039F00894C11CD11CFFEFCF16D104C1F656
:106C500020E090E030E0D50181E0FD0111828F5FFE
:106C600011968830D1F7222309F461C0D5019C9395
:106C7000E32E30FF40C00E94E6338C01F501808195
:106C80008430A1F465E872E0C8010E943437892B92
:106C9000B1F061E872E0C8010E943437892BC9F075
:106CA0006BE772E0C8010E9434371AC08D30F1F4EE
:106CB00065E772E0C8010E943437892B19F4F501A9
:106CC000118219C060E772E0C8010E943437892B35
:106CD00011F481E008C069E672E0C8010E9434370F
:106CE000892B21F482E0F501818305C0C8010E944F
:106CF0008434F5016183E1FE06C00E94E6330E9400
:106D00008434F5016283E2FE15C00E94E6330E94DE
:106D100084346A837B838C839D838D81F501838397
:106D20008C8184838B8185838A81868303C08FEFE6
:106D3000D5018C938501095F1F4F82E090E00E948E
:106D40006E10F501878320E030E0F501E20FF31FBC
:106D5000D8018C919081890F8C932F5F3F4F273002
:106D6000310599F781E090E025960FB6F894DEBFE3
:106D70000FBECDBFDF91CF911F910F91FF90EF908C
:106D8000DF90CF90BF90AF909F908F900895A0E03C
:106D9000B0E0EDECF6E30C942238EC0168817981E7
:106DA0008A819B81611571058105910549F484E211
:106DB000A82E89EDB82E8BE5C82E87E0D82E02C00C
:106DC0005B016C01C601B5012DE133EF41E050E0FC
:106DD0000E94BE3727EA31E440E050E00E948B3742
:106DE0007B018C01C601B5012DE133EF41E050E09C
:106DF0000E94BE37CA01B90124E13BE040E050E007
:106E00000E948B37E61AF70A080B190B17FF08C008
:106E10008FEF9FEFAFEFBFE7E80EF91E0A1F1B1FB2
:106E2000E882F9820A831B838FEF9FEFAFEFBFE702
:106E3000E822F9220A231B23C801B701EAE0CDB7F3
:106E4000DEB70C943E380E94C73608958FE091E07B
:106E50000E94C736089560930F01709310018093CC
:106E60001101909312010895FB01DC018D91813491
:106E70001CF08B350CF4805E659161341CF06B3531
:106E80000CF4605E861B611189F3990B0895FA0179
:106E9000CF93FF93EF93223044F1253234F5C22F84
:106EA000E894CA3049F497FB3EF49095809570952C
:106EB00061957F4F8F4F9F4F2C2F332744275527A6
:106EC000FF93EF930E94D937EF91FF91605D6A3392
:106ED0000CF0695D6193B901CA0160507040804057
:106EE000904051F716F4CDE2C19310828F919F919B
:106EF000CF910C947B37DC01FC01672F71917723D4
:106F0000E1F7329704C07C916D9370836291AE1764
:106F1000BF07C8F30895629FD001739FF001829F5D
:106F2000E00DF11D649FE00DF11D929FF00D839F18
:106F3000F00D749FF00D659FF00D9927729FB00DB5
:106F4000E11DF91F639FB00DE11DF91FBD01CF01C8
:106F500011240895AA1BBB1B51E107C0AA1FBB1F28
:106F6000A617B70710F0A61BB70B881F991F5A95D5
:106F7000A9F780959095BC01CD01089597FB092E46
:106F800005260ED057FD04D014D00AD0001C38F4CA
:106F900050954095309521953F4F4F4F5F4F089545
:106FA000F6F790958095709561957F4F8F4F9F4F25
:106FB0000895A1E21A2EAA1BBB1BFD010DC0AA1F3A
:106FC000BB1FEE1FFF1FA217B307E407F50720F052
:106FD000A21BB30BE40BF50B661F771F881F991FCD
:106FE0001A9469F760957095809590959B01AC0116
:106FF000BD01CF01089591111AC0803219F0895056
:107000008550D0F70895E199FECFBFBBAEBBE09AA3
:1070100011960DB20895E199FECFBFBBAEBB0DBA7C
:1070200011960FB6F894E29AE19A0FBE0895992747
:10703000882708952F923F924F925F926F927F928E
:107040008F929F92AF92BF92CF92DF92EF92FF9278
:107050000F931F93CF93DF93CDB7DEB7CA1BDB0B24
:107060000FB6F894DEBF0FBECDBF09942A883988C9
:1070700048885F846E847D848C849B84AA84B984D0
:10708000C884DF80EE80FD800C811B81AA81B981DC
:10709000CE0FD11D0FB6F894DEBF0FBECDBFED01F0
:0470A0000895FFCF81
:1070A40014141431126E252425841B9C2D8C26BDAA
:1070B40022FC2133217D1FCA1DA51C8E1B3A1BFEF9
:1070C40028822833123512371239125E14A5142A75
:1070D4001533154F15621569150E1A7015691906C1
:1070E40019AA1804263613632814217315AE15BB88
:1070F40015BC15BE15C015C215C415C615C815CACC
:1071040015CC15CE15D015D215D415D615D815DA3B
:1071140015DC15DE15E015E215E415E615E815EAAB
:1071240015EC15DB03E203DC03DD03DE03DF03E020
:1071340003E103EE15F1150116051634182A160994
:10714400183116E017F6188116901646179E160188
:047154000000000037
:00000001FF
